:10000000004000203550000075500000775000007F
:1000100000000000000000000000000000000000E0
:100020000000000000000000000000007950000007
:1000300000000000000000007B5000007D50000028
:100040007F500000E1380000B15400007F500000F4
:100050007F500000000000007F5000007F50000033
:100060007F500000755700007F5000007F50000057
:100070007F5000007F5000007F5000007F50000044
:100080007F5000000D5900007F5000007F5000009D
:100090007F5000007F5000007F5000007F50000024
:1000A0007F5000007F5000000000000000000000B2
:1000B0000000000000000000000000000000000040
:1000C00010B5064C2378002B07D1054B002B02D02E
:1000D000044800E000BF0123237010BD440200204B
:1000E0000000000090B60000044B10B5002B03D0B8
:1000F0000349044800E000BF10BDC04600000000F6
:100100004802002090B60000164B002B00D1144B83
:100110009D46402292029A1A924600218B460F4633
:100120001348144A121A08F032FD0F4B002B00D06E
:1001300098470E4B002B00D0984700200021040068
:100140000D000D48002802D00C4800E000BF08F068
:10015000DDFC2000290005F0C3F908F0B1FCC04621
:100160000000080000400020000000000000000027
:1001700044020020C0250020000000000000000014
:1001800002000120104004D1042A01D9106800099E
:1001900070470020FCE710B50400FFF7F1FF0028CE
:1001A00009D001388000031D22181279002A02D0DC
:1001B00001309842F8D110BD0122096810B51142F2
:1001C00001D0002903DA102000F084F910BD491095
:1001D000062002F011F8F9E7096810B5CB0701D540
:1001E000002903DA102000F075F910BD4910033121
:1001F00089100022052001F0FFFFF6E770B50D68B9
:10020000AB0729D1042D27D90F232A684E68134044
:10021000062B0BD12800FFF7B3FF0123984201DA28
:1002200000200AE09A00AE500133F7E7052B13D106
:10023000F30703D4132000F04DF970BD7610FF2EA4
:10024000F8D82800FFF79CFF2C1D80002018A04242
:10025000E6D926700134FAE70B2000F03BF9DFE71E
:1002600070B50C681120E30712D54D68AB072BD190
:10027000042D29D90F262B6864101E40062E0DD19F
:10028000002C04DD2800FFF77BFFA04203DA1220D8
:1002900000F020F901E0A400605970BD331F012B6C
:1002A00012D82800FFF76CFF8000042E02D128002E
:1002B000FFF771FF002CEADDA042E8DB01202C19DA
:1002C000E3785B001843E8E70B20E1E7F8B501238A
:1002D0000D6811201D4214D003244E6834402CD1E7
:1002E000042E2AD90F2332686D108F681340062B15
:1002F0000ED1002D04DD3000FFF742FFA84203DAE3
:10030000122000F0E7F802E0AD00AF512000F8BD88
:10031000052B12D1002DF3DD3000FFF731FF8000F7
:10032000A842EDDB01231F4201D11320E9E77F1032
:10033000FF2FFAD87519EF70E8E70B20E1E708689E
:1003400010B5830717D1042815D90F23026813406D
:10035000062B03D1FFF714FF430004E0052B05D162
:10036000FFF70EFFC3000120184310BD042B02D17C
:10037000FFF711FFF0E70B2000F0ACF8F5E7000005
:1003800002000120104001D0501070470D22014B97
:100390001A70FAE78402002002000120104004D104
:1003A000042A01D91068000970470020FCE770B5E5
:1003B0000E000400FFF7F0FF05003000FFF7ECFF30
:1003C0000023854206D10434AD0004366519AC42E1
:1003D00002D30123180070BD20783278002801D1A3
:1003E000002AF6D0013401369042F0D00023F1E724
:1003F000F0B585B00393019002912D4E2D4B002A4C
:1004000002D002223270013A00251A601B68F554AE
:10041000019B9D4201DB05B0F0BD029AAB00D058B4
:10042000244B1C68C8239B0037191C1B012318424E
:1004300006D0214A43102100380008F051FF09E09E
:100440001E4A002802D004281BD11D4A2100380072
:1004500008F046FF300008F0A7FF164A039B106023
:10046000002B0CD0019B013BAB4208DD154B9842A1
:1004700005D8431C1360202232540022F254013567
:10048000C6E7042810D90F2302681340042B04D1B7
:1004900001F0EEFE0C4A0300CDE7062B05D1FFF775
:1004A0007BFF0A4A0300C6E70123094AC3E7C046A7
:1004B00085020020A805002035A3000008A3000045
:1004C0000EA300001F03000023AF000013A30000D1
:1004D00024A30000014B1870002070478402002004
:1004E00070B501F0E7FC094C0100251D1F22280012
:1004F00008F061FF280008F057FF0423043080084B
:10050000000118432060200070BDC046600200203A
:10051000C368F0B59D00836889B05D190300183386
:1005200006930369069A9F00069B0390DF194369AF
:1005300001939B00D3180293CD4B1B78002B26D13F
:100540007F222B68CB491C1213409B005B5804355B
:1005500001929F46039B587803F05EFE0023039AA6
:10056000137027E0C24B1B78002B10D12B68019A27
:100570001C121340BF4A9B009B580435E9E7069BB9
:100580003A1DD11ABA4BD82928DD1A221A70039BBA
:10059000B74C9B6821780193EA1A039B92109B78D1
:1005A00012021A43039B587803F03EFE0023039A7D
:1005B00023701370039B069A9B680193ED1A039BAB
:1005C000AD10DD60069BFE1A039BB6101E61029BF8
:1005D0009B1A039A9B10536109B0F0BD1B783C60D5
:1005E000002B01D01700D2E72B6801991C120B4099
:1005F000A0499B005B5817000435AAE7069B3A1DEB
:10060000D11A9B4BD82902DD1A221A70BFE728683D
:100610001B78291D3860002B02D017000D00B6E7AB
:100620006B6801991C120B4092499B005B581700A4
:1006300008358EE7069B3A1DD11A8D4BD82902DD6D
:100640001A221A70A3E7A4001B782C193C60002B17
:1006500001D017009BE72B6801991C120B408549BC
:100660009B005B581700043573E7069B3A1DD11AAF
:100670007F4BD82902DD1A221A7088E77E49A40030
:1006800061581B783960002B01D017007FE72B6879
:1006900001991C120B4077499B005B5817000435E9
:1006A00057E7043F744B3A68A400E250704B1B7844
:1006B000002B00D06BE72B68019A1C1213406D4A87
:1006C0009B009B58043544E76B4BA400E058FFF7B0
:1006D00057FE043F06003868FFF752FE3618012027
:1006E000654B76000643E650614B1B78002B00D02B
:1006F0004DE72B68019A1C1213405E4A9B009B58E1
:10070000043526E7069B3A1DD11A594BD82902DD3C
:100710001A221A703BE70698029C0121A04202D2DD
:1007200021000C3909681B783960002B01D01700B3
:100730002DE72B6801991C120B404E499B005B581A
:100740001700043505E7069B3A1DD11A484BD829F6
:1007500002DD1A221A701AE70699029881420FD216
:1007600003000C3B1B6845495B106418E41AA400A5
:1007700023583B603E4B1B78002B05D0170006E743
:10078000182119700023F4E72B6801991C120B4003
:1007900038499B005B5817000435DAE6069B029A3D
:1007A000934219D213000C3B1B68344A043FA4182F
:1007B0005B10E31A029A39689B0099502C4B1B7806
:1007C000002B00D0E3E62B68019A1C121340294A43
:1007D0009B009B580435BCE61822254B1A70EDE7A8
:1007E000069B029A93422DD2244B3E1FE31814001D
:1007F0000C3C04932368049A5B10D31A029A9B0062
:100800009858FFF7BDFD07903068FFF7B9FD2468E1
:10081000049B64101C1B079BA4001F1801207F0071
:10082000029B0743E7503700114B1B78002B00D089
:10083000ADE62B68019A1C1213400E4A9B009B5890
:10084000043586E618220A4B1A70EDE7069B3A1D1E
:10085000D11A074BD82902DD1A221A7097E602999D
:10086000A40061581B783960002B09D017008EE670
:100870008402002008A1000068230020FDFFFF3F44
:100880002B6801991C120B40D8499B005B5817003C
:1008900004355EE6043F029B3A68A400E250D44B64
:1008A0001B78002B00D072E62B68019A1C121340B3
:1008B000CE4A9B009B5804354BE6029BA4001C19B2
:1008C0002368043F38685E10FFF75AFD3618012090
:1008D000C74B76001B7806432660002B00D056E6F7
:1008E0002B68019A1C121340C04A9B009B58043588
:1008F0002FE6069BA4003F1BBD4CBB420CD82378BF
:10090000002B00D043E62B68019A1C121340B74A13
:100910009B009B5804351CE6B64801F01DFC23786B
:10092000002B00D033E62B68019A1C121340AF4A0B
:100930009B009B5804350CE6A300ED18002C00DA50
:1009400038E6AB4B1B78002B00D020E62B68019AD1
:100950001C121340A54A9B009B580435F9E5043F3F
:100960003B68042B04D1A300ED18002C00DA21E62B
:100970009F4B1B78002B00D009E62B68019A1C12B4
:1009800013409A4A9B009B580435E2E5043F3B68BC
:10099000042B06D0A200AD18002C02DA002B00D1E7
:1009A00008E6934B1B78002B00D0F0E52B68019AEA
:1009B0001C1213408D4A9B009B580435C9E53A1F11
:1009C00013685B10013B002B06DD01215B00A400D6
:1009D0000B432D191360EDE5854B17001B78002B99
:1009E00000D0D4E52B68019A1C1213407F4A9B006B
:1009F0009B580435ADE53A00069B0C32D31AD82B30
:100A000003DD1A227A4B1A70C1E5FF2361005B00F7
:100A10001940FE3BFF3B19433960039906988968EA
:100A2000241204916D1A0399AD1089782D020D439B
:100A300002999D40091A891099401D430B43BB60E0
:100A4000039B7D609C70E4B26B4BE4000292E35820
:100A5000039A9360664A1278002A03D008331D0077
:100A6000029F94E51D00019A9B680C351C121340EF
:100A70005E4A9B009B58029F6BE53B1F1C68029AD5
:100A8000069B93422FD10A20E3070ED4A30715D16A
:100A9000042C13D90F2322681340042B11D12000FA
:100AA00001F0E6FB08F080FC0630643003F09EF8AD
:100AB00000280FD1043D069B02937BE50720042C00
:100AC000F3D02000431E9841FA234042FF331840E0
:100AD0000730EAE7039B2100587803F0B7FB0023B7
:100AE000039A1370E7E7029B029A0C3B1B68039979
:100AF0005B109B00D31A0C3B1C601F1D1300083BAE
:100B00001B685A108A70D2B23B49D2005B0055581C
:100B10009B0A039A9B009560ED18029B069A043B82
:100B20001B685B109B00D3180293314B1B78002B82
:100B300000D02CE52B68019A1C1213402B4A9B0015
:100B40009B58043505E53B1F1868FFF719FCA40006
:100B500006003F1B1E2827DC00280DDC244B1B78D9
:100B6000002B00D013E52B68019A1C1213401F4A7A
:100B70009B009B580435ECE401F08AF9033E3618DB
:100B800001F086F91D4B801B9842F9D8184B1B7851
:100B9000002B00D0FBE42B68019A1C121340134A6F
:100BA0009B009B580435D4E40123039A137001F091
:100BB0006FF9039B0A3886195E60FBE43B1F1868D7
:100BC000FFF7DEFBA40006003F1B002818DC084BE3
:100BD0001B78002B00D0DAE42B68019A1C1213401A
:100BE000024A9B009B580435B3E4C04608A10000AC
:100BF0008402002038A30000701B00209F860100A3
:100C0000C64B984203DD1D22C54B1A70BFE4012379
:100C1000039A137001F03CF9FA239B005E43039B97
:100C20000A3E30185860C5E4A300FF1A00232000D4
:100C30001A003900FFF7DCFBBA4EBB4C31682000CC
:100C400003F0BCF93168200003F007FB3168200095
:100C500001F0A4FBB24B1B78002B00D097E42B686B
:100C6000019A1C121340B14A9B009B58043570E452
:100C7000AB4BA4001B783F1B002B00D087E42B68F4
:100C8000019A1C121340A94A9B009B58043560E44A
:100C9000039803F00FF8A24B1B78002B00D076E4EA
:100CA0002B68019A1C121340A04A9B009B580435E4
:100CB0004FE43B1F1868002838D1083B1868C30769
:100CC0001ED540103A0001234100083A0B4313603F
:100CD000002859DD01234200391F1A430A603A00F7
:100CE000083A12681A41101A3A000C3A116819426F
:100CF0001FD0C0189840A4001843029BE05027E082
:100D000083070FD104280DD90F2302681340062B47
:100D100002D1FFF741FBD5E7052B03D1FFF73CFBE1
:100D20008000CFE719227E4B1A7030E44010013862
:100D3000CEE78A0723D1042921D90F220E68324039
:100D4000062A15D1013080004358029AA400A3500E
:100D5000734B1B78002B01D0FFF719FC2B68019A0D
:100D60001C121340714A9B009B580435FFF7F1FB9E
:100D7000052A04D108180079A4004000BCE7192214
:100D8000674B1A70FFF703FC0435E1E7A300069AEE
:100D9000FB189B1AD82B13DC0122631E002C14DCD9
:100DA0005F4B1B78002B01D0FFF7F1FB2B68019AFA
:100DB0001C1213405D4A9B009B580435FFF7C9FB8A
:100DC0001A22574B1A70FFF7E2FB3A601C000437F7
:100DD000E3E7069A3B1D9B1A514ED82B03DD1A23DD
:100DE0003370FFF7D4FB069B029AA40093422AD2E9
:100DF0003B1F1868FFF7C4FA011E21DD029B0C3B64
:100E00001A68521082421BDB9007801A484B401828
:100E1000C018029B8000C2583B1B1A60404B3F1B0E
:100E20001B780437002B01D0FFF7B1FB2B68019A28
:100E30001C1213403D4A9B009B580435FFF789FB69
:100E400020233370EAE71823FBE7A3009C46FE1A31
:100E5000002C17DC1C22324B1A70002333606346CF
:100E6000FF1A2F4B04371B78002B01D0FFF78FFBA5
:100E70002B68019A1C1213402C4A9B009B58043586
:100E8000FFF767FB002033685A108300F1580123F5
:100E90000B4003D10D21224A1170DFE749108A422D
:100EA00000DD0A0001308442EFDC012352001343CD
:100EB000D4E7A3009C46FE1A002C17DC1C22184B1A
:100EC0001A70002333606346FF1A154B04371B78F2
:100ED000002B01D0FFF75BFB2B68019A1C1213401B
:100EE000124A9B009B580435FFF733FB0020336800
:100EF0005A108300F15801230B4003D10D21084AF9
:100F00001170DFE749108A4200DA0A00013084429A
:100F1000EFDC012352001343D4E7C04680EE3600D5
:100F200084020020A80500208502002008A10000FE
:100F3000FCFFFF3F3B00083B1868FFF721FA3B1F0F
:100F400006001868FFF71CFA0023864200DA043313
:100F5000A4003A1B17001360E34B04371B78002BE7
:100F600001D0FFF714FB2B68019A1C121340DF4AD3
:100F70009B009B580435FFF7ECFA3B00083B1868D0
:100F8000FFF7FEF93B1F06001868FFF7F9F9F30FAA
:100F9000C217B0425341A4003A1B17009B001360D4
:100FA000D14B04371B78002B01D0FFF7F0FA2B68E8
:100FB000019A1C121340CD4A9B009B580435FFF741
:100FC000C8FA3B00083B18683B1F1968A600BE1B07
:100FD0000423814202D0042802D8002333601CE09D
:100FE0000123184201D01942F7D103239C4618422D
:100FF000F3D102680C331A40042AEED16246114242
:10100000EBD10429E9D90A681340042BE5D1FFF795
:10101000CEF9431E984180003060B34BA4001B788A
:101020003F1B0437002B01D0FFF7B1FA2B68019A60
:101030001C121340AD4A9B009B580435FFF789FAF8
:101040003B00083B18683B1F1968A600BE1B002325
:10105000814202D0042802D8042333601CE001231B
:10106000184201D01942F7D103239C461842F3D10C
:1010700002680C331A40042AEED162461142EBD1C9
:101080000429E9D90A681340042BE5D1FFF78FF949
:101090004342584180003060934BA4001B783F1BB3
:1010A0000437002B01D0FFF772FA2B68019A1C124B
:1010B00013408E4A9B009B580435FFF74AFA3B00C9
:1010C000083B1868FFF75CF93B1F06001868FFF73C
:1010D00057F9F317C20F86425341A4003A1B170079
:1010E0009B001360804B04371B78002B01D0FFF767
:1010F0004EFA2B68019A1C1213407C4A9B009B58A5
:101100000435FFF726FA3B00083B1868FFF738F96B
:101110003B1F06001868FFF733F90023864200DD05
:101120000433A4003A1B170013606F4B04371B787D
:10113000002B01D0FFF72BFA2B68019A1C121340E9
:101140006A4A9B009B580435FFF703FA3B1F1B6854
:10115000A400043B5A1E93413A1B17009B001360E6
:10116000614B04371B78002B01D0FFF710FA2B6876
:10117000019A1C1213405D4A9B009B580435FFF7EF
:10118000E8F93B00083B1868FFF7FAF83B1F060038
:101190001868FFF7F5F832180120A4003B1B1F0068
:1011A000520002431A60504B04371B78002B01D0C9
:1011B000FFF7EDF92B68019A1C1213404B4A9B0074
:1011C0009B580435FFF7C5F93B00083B1868FFF74B
:1011D000D7F83B1F06001868FFF7D2F8321A012033
:1011E000A4003B1B1F00520002431A603E4B043711
:1011F0001B78002B01D0FFF7CAF92B68019A1C124B
:1012000013403A4A9B009B580435FFF7A2F93B0074
:10121000083B1868FFF7B4F83B1F06001868FFF793
:10122000AFF802000120A4003B1B1F0072435200D4
:1012300002431A602C4B04371B78002B01D0FFF7B8
:10124000A6F92B68019A1C121340284A9B009B5850
:101250000435FFF77EF93B1F1868FFF791F8061E6B
:1012600017D11F22204B1A70A4003B1B1F001E60C9
:101270001D4B04371B78002B01D0FFF788F92B6832
:10128000019A1C121340194A9B009B580435FFF722
:1012900060F93B00083B1868FFF772F8310005F071
:1012A00055FE012640000643DEE73B1F1868FFF7A6
:1012B00067F8061E1CD11F220B4B1A70A4003B1BA3
:1012C0001F001E60084B04371B78002B01D0FFF76E
:1012D0005EF92B68019A1C121340044A9B009B582C
:1012E0000435FFF736F9C0468402002008A100004B
:1012F0003B00083B1868FFF743F8310005F00CFF8E
:10130000012649000E43D9E73B1F1868FFF738F85C
:10131000C217801850400122A4003B1B1F00400050
:1013200010431860F14B04371B78002B01D0FFF7F6
:101330002EF92B68019A1C121340ED4A9B009B5812
:101340000435FFF706F9A300FE1A3068012C24D1FA
:10135000FFF716F80494079007F07EFF079900291D
:1013600000DC012105F0D8FE049BA400C91801236C
:1013700049001943DD4B3F1B1B7831600437002BBC
:1013800001D0FFF704F92B68019A1C121340D84AC8
:101390009B009B580435FFF7DCF8FEF7F1FF049043
:1013A0007068FEF7EDFF049B0130C31A0793D3E783
:1013B000A300FE1A31002000049300F08FFF049B6D
:1013C0003060FF1AC94B04371B78002B01D0FFF7A0
:1013D000DEF82B68019A1C121340C54A9B009B58EB
:1013E0000435FFF7B6F83B00083B1868FEF7C8FF66
:1013F0003B1F06001868FEF7C3FF02000120A4008F
:101400003B1B1F003240520002431A60B74B0437A7
:101410001B78002B01D0FFF7BAF82B68019A1C1239
:101420001340B34A9B009B580435FFF792F83B00EA
:10143000083B1868FEF7A4FF06003B1F1868FEF77C
:101440009FFF320002430120A4003B1B1F005200FB
:1014500002431A60A54B04371B78002B01D0FFF71D
:1014600096F82B68019A1C121340A14A9B009B58C6
:101470000435FFF76EF83B00083B1868FEF780FF65
:1014800006003B1F1868FEF77BFF32004240012038
:10149000A4003B1B1F00520002431A60934B043709
:1014A0001B78002B01D0FFF772F82B68019A1C12F1
:1014B00013408F4A9B009B580435FFF74AF83B1FA7
:1014C0001868FEF75DFFC0430122A4003B1B1F000C
:1014D000400010431860854B04371B78002B01D067
:1014E000FFF755F82B68019A1C121340804A9B00A5
:1014F0009B580435FFF72DF83B00083B1868FEF7B2
:101500003FFF06003B1F1868FEF73AFF320082409B
:1015100051000122A4003B1B1F000A431A60734BB9
:1015200004371B78002B01D0FFF731F82B68019AA4
:101530001C1213406E4A9B009B580435FFF709F8B4
:101540003B00083B1868FEF71BFF06003B1F1868AE
:10155000FEF716FF3200024151000122A4003B1B9E
:101560001F000A431A60614B04371B78002B01D01F
:10157000FFF70DF82B68019A1C1213405C4A9B0080
:101580009B580435FEF7E5FF3B000C3B1868FEF75F
:10159000F7FE3B00083B06001868FEF7F1FEF11766
:1015A0000200C317300005F009FE3B1F04900591AF
:1015B0001868FEF7E5FE02000498059905F0B2FDF3
:1015C00043000120A4003E1B37001843474B306006
:1015D0001B780437002B01D0FEF7D9FF2B68019A46
:1015E0001C121340424A9B009B580435FEF7B1FF82
:1015F000A300FE1A310020000493FEF7DDFD049BDA
:101600003060FF1A394B04371B78002B01D0FEF7EE
:10161000BEFF2B68019A1C121340354A9B009B5851
:101620000435FEF796FFA300FE1A31002000049354
:10163000FEF7D2FD049B3060FF1A2C4B04371B7859
:10164000002B01D0FEF7A3FF2B68019A1C12134058
:10165000274A9B009B580435FEF77BFFA300FF1A27
:1016600039002000FEF7CAFD204B1B78002B01D06B
:10167000FEF78DFF2B68019A1C1213401C4A9B0039
:101680009B580435FEF765FFA300FE1A31002000C9
:101690000493FEF7E5FD049B3060FF1A134B0437FB
:1016A0001B78002B01D0FEF772FF2B68019A1C12E9
:1016B00013400F4A9B009B580435FEF74AFFA300D6
:1016C000FF1A39002000FEF701FE084B1B78002BA3
:1016D00001D0FEF75CFF2B68019A1C121340044AEC
:1016E0009B009B580435FEF734FFC046840200205F
:1016F00008A10000A300FE1A310020000493FEF7A9
:101700001EFE049B3060FF1AF14B04371B78002B40
:1017100001D0FEF73CFF2B68019A1C121340ED4AE2
:101720009B009B580435FEF714FF069B3E1DF31AE1
:10173000E74CD82B03DD1A232370FEF728FF00F0B7
:10174000B1FB43000120184323783860002B02D0FE
:101750003700FEF71CFF2B68019A1C121340DD4A6C
:101760009B009B5837000435FEF7F3FE069B3E1D99
:10177000F31AD74CD82B03DD1A232370FEF707FF8B
:1017800000F086FBD44B4000184001231843237817
:101790003860002B02D03700FEF7F9FE2B68019A63
:1017A0001C121340CB4A9B009B5837000435FEF7B0
:1017B000D0FE0123A600BE1B20001A003100FEF758
:1017C00017FEC64C2068643002F010FA002802D1DF
:1017D000043DFEF7EFFE039B21685A78C04802F0F3
:1017E0004AFD0123039A3700137000F051FBBD4BF3
:1017F00022681B68063253431818039B5860FEF793
:10180000D9FEA600BE1B2000012300223100FEF7F6
:10181000EFFDB24C2068643002F0E8F90028D7D020
:10182000AF4802F023FBDCE7A4003E1BFEF758FEA6
:101830003700A74B30601B780437002B01D0FEF730
:10184000A6FE2B68019A1C121340A24A9B009B58CB
:101850000435FEF77EFEA4003E1B300000F050FB76
:1018600037009B4B30601B780437002B01D0FEF70C
:101870008EFE2B68019A1C121340964A9B009B58BF
:101880000435FEF766FEA4003E1B300000F03AFB74
:1018900037008F4B30601B780437002B01D0FEF7E8
:1018A00076FE2B68019A1C1213408A4A9B009B58B3
:1018B0000435FEF74EFEA4003E1B300000F024FB72
:1018C0003700834B30601B780437002B01D0FEF7C4
:1018D0005EFE2B68019A1C1213407E4A9B009B58A7
:1018E0000435FEF736FEA4003F1B380000F02AFB4B
:1018F000774B1B78002B01D0FEF749FE2B68019A2D
:101900001C121340734A9B009B580435FEF721FEBE
:10191000A300FE1A31002000049300F033FB049B67
:101920003060FF1A6A4B04371B78002B01D0FEF79A
:101930002EFE2B68019A1C121340664A9B009B588E
:101940000435FEF706FEA4003F1B380000F054FBF0
:101950005F4B1B78002B01D0FEF719FE2B68019A14
:101960001C1213405B4A9B009B580435FEF7F1FDA7
:101970000121200000F028FB554B1B78002B01D0E3
:10198000FEF705FE2B68019A1C121340514A9B007A
:101990009B580435FEF7DDFD0021200000F014FB0C
:1019A0004B4B1B78002B01D0FEF7F1FD2B68019A01
:1019B0001C121340474A9B009B580435FEF7C9FD93
:1019C000A4003E1B300000F033FB3700404B30607A
:1019D0001B780437002B01D0FEF7D9FD2B68019A44
:1019E0001C1213403B4A9B009B580435FEF7B1FD87
:1019F000A4003E1B300000F02FFB3700344B30605A
:101A00001B780437002B01D0FEF7C1FD2B68019A2B
:101A10001C1213402F4A9B009B580435FEF799FD7A
:101A2000A4003F1B380000F0F1FA294B1B78002B73
:101A300001D0FEF7ACFD2B68019A1C121340254A19
:101A40009B009B580435FEF784FDA4003F1B380023
:101A500002F0BEFE1E4B1B78002B01D0FEF797FD57
:101A60002B68019A1C1213401A4A9B009B5804359C
:101A7000FEF76FFDA4003E1B300002F051FF37005F
:101A8000134B30601B780437002B01D0FEF77FFD2D
:101A90002B68019A1C1213400E4A9B009B58043578
:101AA000FEF757FDA4003F1B380002F061FE084B13
:101AB0001B78002B01D0FEF76AFD2B68019A1C12DF
:101AC0001340044A9B009B580435FEF742FDC04674
:101AD0008402002008A10000FEFFFF7FA80500206F
:101AE0008502002004000020A4003E1B300002F00C
:101AF00055FE3700B14B30601B780437002B01D006
:101B0000FEF745FD2B68019A1C121340AC4A9B005E
:101B10009B580435FEF71DFDA300FF1A3900200075
:101B200000F0B0FEA54B1B78002B01D0FEF72FFD77
:101B30002B68019A1C121340A14A9B009B58043544
:101B4000FEF707FDA300FF1A3900200000F024FD76
:101B50009A4B1B78002B01D0FEF719FD2B68019AD8
:101B60001C121340964A9B009B580435FEF7F1FC6B
:101B7000A300FF1A3900200000F01EFD8F4B1B78D8
:101B8000002B01D0FEF703FD2B68019A1C121340B5
:101B90008B4A9B009B580435FEF7DBFCA300FF1A21
:101BA0003900200000F030FD844B1B78002B01D061
:101BB000FEF7EDFC2B68019A1C121340804A9B0033
:101BC0009B580435FEF7C5FCA300FE1A3100200027
:101BD000049302F0E7FE049B3060FF1A774B043752
:101BE0001B78002B01D0FEF7D2FC2B68019A1C1247
:101BF0001340734A9B009B580435FEF7AAFCA300D0
:101C0000FE1A31002000049302F0E4FE049B3060D1
:101C1000FF1A6A4B04371B78002B01D0FEF7B7FC84
:101C20002B68019A1C121340654A9B009B5804358F
:101C3000FEF78FFCA300FE1A31002000049302F08F
:101C40008AFE049B3060FF1A5C4B04371B78002B24
:101C500001D0FEF79CFC2B68019A1C121340584AD5
:101C60009B009B580435FEF774FCA300FE1A31005C
:101C70002000049302F088FE049B3060FF1A4F4B53
:101C800004371B78002B01D0FEF781FC2B68019AEA
:101C90001C1213404A4A9B009B580435FEF759FC1E
:101CA000A300FF1A3900200000F08EFD434B1B7883
:101CB000002B01D0FEF76BFC2B68019A1C1213401D
:101CC0003F4A9B009B580435FEF743FCA300FF1AD4
:101CD0003900200000F0C0FC384B1B78002B01D0ED
:101CE000FEF755FC2B68019A1C121340344A9B00E6
:101CF0009B580435FEF72DFCA300FE1A310020008E
:101D0000049300F0D5FD049B3060FF1A2B4B043781
:101D10001B78002B01D0FEF73AFC2B68019A1C12AD
:101D20001340274A9B009B580435FEF712FCA30082
:101D3000FF1A3900200000F02FFD204B1B78002BEC
:101D400001D0FEF724FC2B68019A1C1213401C4A98
:101D50009B009B580435FEF7FCFBA300FF1A3900DB
:101D6000200001F0C9FE154B1B78002B01D0FEF7B7
:101D70000EFC2B68019A1C121340114A9B009B58C1
:101D80000435FEF7E6FBA300FE1A310020000493A1
:101D900001F0B2FE049B3060FF1A084B04371B7839
:101DA000002B01D0FEF7F3FB2B68019A1C121340A5
:101DB000034A9B009B580435FEF7CBFB84020020AE
:101DC00008A100000023F7B55A1E0192002B07DA84
:101DD00000F0A2FD02F04CF902F0A4FA6423019392
:101DE00000263000194B1968B14212DD184B1A68F1
:101DF00001328A420FDAF0241A601D68154F6C43D5
:101E0000E35D002B1FD0E419022B06D12000FEF762
:101E10007FFB019BD8E70022EDE7012B0DD10028C5
:101E200001D100F035F8F0226A43BB185B680A491B
:101E3000C31A8B4201D80223BB54F0235D43054BE8
:101E4000EB5C022BE2D00136CCE7C046AC050020AB
:101E500000000020101200209F8601000020704723
:101E600000207047002070470020704701220020AA
:101E7000054B06491A615850043103305850083157
:101E8000801858501A607047008000400405000018
:101E90000122034B1A64A822D20098587047C0460A
:101EA0000080004010B5FFF7F3FFFA21890004F02D
:101EB000C3FF10BD0048704788A300001A20704778
:101EC00070B5054E0400335C0D008B4202D003F068
:101ED0009DFC355570BDC046B005002070B500248E
:101EE000064D635D012B05D10021200003F08EFC1F
:101EF0000023635501341A2CF2D170BDB0050020C7
:101F00000D20704735207047036870B55B100120C5
:101F1000052B12D8094A9B009C58094D2B5D002BBC
:101F200005D00021200003F071FC00232B55200078
:101F300003F01AFB43000120184370BD70A300009A
:101F4000B0050020036870B55D10192D14D80B4E34
:101F50004468735D012B05D00121280003F056FC75
:101F600001237355064964108C4202DCE143C91712
:101F70002140280003F07EFB70BDC046B005002064
:101F8000FF0300000B6870B55D10192D16D80024F2
:101F9000012804DD4C68043C63425C416400094E46
:101FA000735DA34204D02100280003F02FFC745578
:101FB000280003F05FFC0423012800D00023180050
:101FC00070BDC046B005002070B504000D00192892
:101FD0000ED8084E335C012B04D0012103F016FC0F
:101FE00001233355290020004D1EA94103F02CFC8C
:101FF00070BDC046B005002010B543680068191FC9
:102000004B4259414010FFF7DFFF10BD37B569461D
:102010000A00064B30CB30C203680220042B02D1E9
:1020200000F0CAFA37BD00F0EFFAFBE748A3000062
:1020300010B5084C237D002B05D00021142003F09F
:10204000E5FB00232375142003F014FC43425841A0
:10205000800010BDB005002010B5084CA37D002BFA
:1020600005D00021162003F0D1FB0023A375162014
:1020700003F000FC43425841800010BDB005002031
:102080007047704710B5034A0421034801F020FD52
:1020900010BDC04650A300005CAA0000E12110B5AD
:1020A0004902094803F05EF8FFF7E0FE0A2003F05A
:1020B00055FA0023FF21054A995401331A2BFBD10D
:1020C00000F076FD10BDC04698110020B00500203C
:1020D000F8B50B4E070030000D0003F08BF804003C
:1020E000A84200DD2C003D00EB1B9C4205DD3000CA
:1020F00003F08AF828700135F6E72000F8BDC046E5
:102100009811002010B50100014803F033F810BD0C
:102110009811002010B5054C200003F039F8E1219A
:102120002000490203F01EF810BDC046981100209F
:10213000064B01201A68064B06491A6000239A00D4
:1021400001338850642BFAD17047C046D405002073
:10215000CC0500206823002000B59BB00200054993
:1021600001A807F0EFF801A801F09CFE02F0DAF8F0
:10217000FCE7C0460EA4000037B5184D04002868DF
:10218000002801D006F0F0FCA400200006F0E2FCDC
:102190002860002802D11248FFF7DEFF01AB984209
:1021A00007D2104B02196B440193934201D20E489F
:1021B000F2E7042802D808302860083C2B680B4A54
:1021C0001C1913600A4B01201C60002309499A0066
:1021D00001338850642BFAD137BDC046D4050020A6
:1021E000B4A300001CFCFFFFE4A30000CC0500200A
:1021F000D00500206823002070B50D4D0D4E040061
:102200004B1C28689B003668C318B34203D90A20C8
:10221000FEF760F970BD2B600500AB4205D80F23B7
:1022200009011C4021430160F4E704C5F5E7C046FD
:10223000CC050020D00500200322CB1C70B50C007B
:10224000D9171140C9180500891000220420FFF792
:10225000D3FF0023A34206DBE343DB171C4000232C
:102260000419237170BDE95CC21811710133F1E7E3
:1022700010B5830706D1042804D90F2208C81340DB
:10228000042B03D00E20FEF725F9014810BDC046EF
:102290001EA4000010B501240B681C4016D05C1071
:1022A000200005F0E7F80B4904F0B2FF06F07AFBD6
:1022B00003F024FC0022084B05F04AFD03F0C6FBA6
:1022C00006F000FB43000120184310BD0D20FEF76F
:1022D00001F9E5E7D30237390000D04010B50324F7
:1022E0000868044006D1042804D90F23026813406B
:1022F000042B03D00E20FEF7EDF810BDFFF7B8FF5A
:1023000003782100233B5A4253411022C01807F0A2
:10231000E9F880239B05C218044B9A4201D9142086
:10232000E9E7430001201843E7E7C046FFFFFF3F0E
:1023300010B5034A0221034801F0CAFB10BDC04694
:1023400024A400001FA400000020704710B51E2028
:10235000FEF7C0F810BD10B51E20FEF7BBF810BD8B
:1023600010B51E20FEF7B6F810BD10B51E20FEF702
:10237000B1F810BD10B51E20FEF7ACF810BD10B5B9
:102380001E20FEF7A7F810BD10B51E20FEF7A2F81C
:1023900010BD10B51E20FEF79DF810BD704700005F
:1023A00010B5034A0921034801F092FB10BDC04655
:1023B00044A400008CA400000120034B1860034BD0
:1023C0001B68834018437047EC050020D8050020A7
:1023D000F0B5EFF310810123194083F31088134CFB
:1023E000134AA4461268134E013A9340124F134AFF
:1023F000002B17D0146803420FD03D682C60C046F4
:10240000C046C046C046C046C046C046C0460C4C4A
:102410001568246825605B08EAE765462C60146847
:102420003460F8E781F31088F0BDC046080500501D
:10243000080000200C050050F8050020F4050020DD
:10244000F005002030B585B001AD0C22064928000A
:1024500006F094FB0024285D01210134FFF730FDD4
:102460000C2CF8D105B030BD18A50000F0B585B032
:102470006A463C4B3C4913800F2301AF93700C31EB
:102480000922380006F07AFBFFF70CFD374B384D78
:10249000C0182B68984201D200232B602C68002CB6
:1024A00044D13E5D01213000FFF70AFD01340121D6
:1024B000300003F0C9F9092CF3D100246B461E5DEE
:1024C00001213000FFF7FCFC01340021300003F053
:1024D000BBF9032CF2D1C82080000138C046C046A9
:1024E000C046C046C046C046C046C046C046C046BC
:1024F000C046C046F1D100210520FFF7E1FC6B4644
:1025000000211878FFF7DCFC6B4600215878FFF7B4
:10251000D7FC6B4600219878FFF7D2FCFFF7C2FC8E
:10252000002413302860200005B0F0BDFFF7BAFC8E
:102530002B6800249842F6D3052003F015F80D4BC4
:102540000D4EC0180BD430603068032104F0FEFC3F
:1025500000230A4A30602B6013600124E3E73460F3
:10256000F2E7C0460D0E000018A50000102700007D
:10257000E4050020C8FEFFFFD8050020EC05002080
:1025800010B50124044002D04410200010BD0D20DD
:10259000FDF7A0FFF9E700000022054B10B51A6017
:1025A000044B1B68934201D002F08AFA002010BD50
:1025B000E8050020BC10002070B508680D00FFF78A
:1025C000DFFF04006868FFF7DBFF621E0100042ADA
:1025D00014D8451E042D11D805236B439B180122E6
:1025E00015009D402B00064805682B430360054BF2
:1025F0001B68002B02D0200002F063FA002070BD9F
:10260000E8050020BC10002070B508680D00FFF739
:10261000B7FF04006868FFF7B3FF621E0100042AD9
:1026200013D8451E042D10D805236B439B18012297
:102630009A400748036893430360064B1B68002BCE
:1026400003D00022200002F03CFA002070BDC046FA
:10265000E8050020BC100020F0B5050089B008682E
:102660000C00FFF78DFF0690022D36DD6068FFF746
:1026700087FF0190A068FFF783FF04000127231D57
:10268000661E0793731C0293079B9E4235D0052359
:1026900073430593019B019D05330493049BAB4257
:1026A0001ED0042E16D86B1E042B13D80122059BB6
:1026B0002349013B5B199A409446224A0B681068F3
:1026C000069A3A4003920DD062461A430A600122EC
:1026D00000280DD17F000135E0E701240194CDE70A
:1026E000029ECFE7624693430B600028F2D0039A24
:1026F0000299280002F0E5F9ECE7019B1E1D042E6B
:102700001AD8012C18D1002505273B0021006B4366
:102710009B1999400B000A4A013511689943094BEE
:1027200011601B68002B05D0019B0022581D290059
:1027300002F0C7F9052DE8D1002009B0F0BDC04670
:10274000E8050020BC10002010B5041E10DA1A2481
:102750000A4BA400E25801239340094A0949136037
:10276000094A1160094A0A4911600A4A136010BDFA
:10277000FFF7A4FBA042EADDEAE7C0469CB10000F7
:10278000F405002008050050F8050020F0050020A1
:102790000C050050180500500200086810B5C3076A
:1027A0000DD540101823012A03DD4A68042A00D100
:1027B0000833044A1360FFF7C7FF002010BD012053
:1027C0004042EFE7080000202B4BF7B51B680C00D8
:1027D000002B03D101204042FFF7B6FF01262468F9
:1027E00034421AD0FF226310120260121040DAB293
:1027F0001043FF221B021204134018431F4B1B6897
:10280000202B06D1B4401E4BA40EA400E3580002B6
:102810001843FFF7DDFD0020FEBD03252540FAD15A
:10282000042CF8D90F2322681340062BF3D1FF277D
:10283000130901933F02019B9D42ECDA0135AB0085
:10284000E3583342F7D05A105812D1B238400843F7
:10285000FF21120209040A401043084A1268202A84
:1028600006D15B009B0E06499B000202585810439C
:10287000FFF7AEFDDFE7C046F405002008000020AA
:1028800008A70000086810B5C30703D5FFF778FE56
:10289000054B1860054B1B68002B03D0024B1868D2
:1028A00002F010F9002010BDE8050020BC10002047
:1028B0000868F8B5C3071AD5FFF762FE0300203B8E
:1028C0005E2B25D80520012258430023114E451DBB
:1028D000A84219D005211024375C3C4200D09B1837
:1028E0000139520064100029F7D10130F0E7830765
:1028F0000ED104280CD90F2203681A40042A07D1EC
:102900001B0905D00079D9E701205B001843F8BD09
:102910000120FCE72DA500007FB5A04C2368002B0B
:102920000AD19F4A1268002A06D19E4B1B68002BD1
:1029300001D0FFF79BFD7FBD9B4D2A68002A26D161
:10294000984A1268002A1BD0FFF790FD0028F2D0A9
:10295000FFF778FD924B24681A681C60002A16D095
:10296000002C14D101AD0C229049280006F006F984
:10297000285D00210134FFF7A3FA0C2CF8D1DAE727
:10298000874A1268002AE5D1002BE3D0E0E7002156
:102990000D2002F059FF00210E2002F055FF00210A
:1029A0000F2002F051FF2E68012E5DD0022E00D1C3
:1029B000A2E0002E51D101363100794C0420236869
:1029C000994302F041FF04212368052019404B423E
:1029D000594102F039FF10212368062019404B426B
:1029E000594102F031FF80212368090119404B420F
:1029F00059410C2002F028FF802123680902194068
:102A00004B4259410B2002F01FFF802123684902ED
:102A100019404B4259410A2002F016FF80212368D9
:102A2000890219404B425941092002F00DFF8021D3
:102A30002368C90219404B425941082002F004FFA3
:102A4000802321681B0319404B425941072002F0A3
:102A5000FBFE31000D2002F0F7FE2B680321581C0D
:102A600004F05AFB296066E702214D4C07202368D9
:102A700019404B42594102F0E7FE0820216801400D
:102A80004B42594102F0E0FE80212368C900194001
:102A90004B425941052002F0D7FE802123684901AD
:102AA00019404B425941062002F0CEFE8021236896
:102AB000C90119404B425941042002F0C5FE802152
:102AC0002368890319404B4259410A2002F0BCFE99
:102AD000802321681B0419404B425941092002F010
:102AE000B3FE31000C2002F0AFFE31000B2002F0EB
:102AF000ABFE31000E20AEE72021294C07202368D1
:102B000019404B42594102F09FFE402123680820A2
:102B100019404B42594102F097FE80212368092059
:102B200019404B42594102F08FFE80212368490031
:102B300019404B4259410A2002F086FE8021236849
:102B4000890019404B4259410B2002F07DFE802143
:102B50002368890119404B4259410C2002F074FE50
:102B600080212368490319404B425941062002F055
:102B70006BFE80212368C90319404B425941042050
:102B800002F062FE802321685B0419404B425941E8
:102B9000052002F059FE01210F205CE7E805002026
:102BA000E0050020EC050020DC05002018A5000051
:102BB000012010B54042FFF7C7FD0020FFF708FCD9
:102BC00010BD000010B5034A0921034800F080FF42
:102BD00010BDC04608A8000050A8000030B502246F
:102BE0008025094B094AED009C505C59002CFCD013
:102BF000A124E400884202D30021995030BD8025F1
:102C0000ED0018514019F5E700E00140040500000F
:102C100010B5002806D1C020B02140028902FFF77C
:102C2000DDFF10BDB02080218002C902F7E700005F
:102C300043425841064B40421840B0239B02C01803
:102C4000036800201A0E532A01D11B02180A70478C
:102C500000C0FEFF30B501248025054B054AED007C
:102C60009C505C59002CFCD001600021995030BD73
:102C700000E001400405000043425841074B404238
:102C80001840B0239B02C018A62310B50902DB052B
:102C9000090A1943FFF7DEFF10BDC04600C0FEFF62
:102CA00070B5012480250D4B0D4EED009C515C59F3
:102CB000002CFCD0002902DC00229A5170BD55780E
:102CC00014782D0225439478013924042543D478BF
:102CD000043224062C4310C0ECE7C04600E001405B
:102CE0000405000070B505004B680A009C1C21001B
:102CF000A400FFF7D5FF281970BD0000134B1B6817
:102D0000002B0CD08022B023D2029B0200280BD1D2
:102D10001A1D5B681B0E522B00D110007047B022A9
:102D2000C02392025B02F1E782420DD903681B0EB9
:102D3000522B09D1436802339B00C018824203D949
:102D400003681B0E522BE9D00020E7E7FC060020A9
:102D500070B50020FFF7D2FFFF260500002801D143
:102D6000280070BD03681C143440FFF7C7FFDA2C3D
:102D7000F4D10500F2E700008022F0B55200A1B0C6
:102D80000021674805F003FF8022002152006548BA
:102D900005F0FDFE644BFF271B681A0004935342A5
:102DA0005A4110000592FFF733FF049C0020631E78
:102DB0009C415E4B64421C405D4BE418FFF7C8FF2A
:102DC0000600002E2DD10498FFF732FF411C059814
:102DD000FFF752FF059A574D534B2C601A60FFF7CF
:102DE00099F9514B64201B68A0215A4253414F4A24
:102DF0005B421340B0222C6892029B18E41A604395
:102E0000490204F0A3F8A0225202030000924A49AA
:102E1000220007A806F096FA07A801F043F821B0AF
:102E2000F0BD3268131412123A403B4003921A006C
:102E30000A3A092A49D83A4B039A995C002931D1B8
:102E400010223E4805F0A3FE35002B6803991A12A4
:102E50003A40914209D11A143A400B2A27D0132A3A
:102E60002DD00A2A01D1354B1D602800FFF746FFFF
:102E7000051EEAD1314B196800290FD02000FFF759
:102E800031FF04002D4B5B195968002903D0200045
:102E9000FFF728FF040004350C2DF3D1204B01214E
:102EA000039A99543000FFF729FF060089E73B4059
:102EB000022BDADC214A9B00D3185D60D5E7102293
:102EC00000211E4805F063FECFE71A00153A082AD4
:102ED000E8D8144A0399525C002AE3D13500152B37
:102EE00000D01500300003681A143A40152A0FD09C
:102EF0001D2A00D10025FFF701FF0028F3D1002D86
:102F000004D020002900FFF7EDFE0400054BC6E7C2
:102F1000039A1B123B409A42EDD10500EBE7C046F5
:102F2000FC05002004070020FC06002000C0FEFF76
:102F300004C0020000070020E9A80000F8240020D7
:102F4000F0B50020B7B00024FFF7D8FE2700050039
:102F50002600002D2ED1284D2868FFF769FE32008B
:102F60003B0001900094254904A806F0EBF904A861
:102F700000F098FF224B64201C682B68A0215A4265
:102F80005341204A5B421340B02292029B18E41A3C
:102F90006043490203F0DAFFA022520203000092CC
:102FA0001949220004A806F0CDF904A800F07AFF20
:102FB00037B0F0BDFF226B6829689C460233FF18CA
:102FC0000B12013613409C4200DA1C00FF200A1449
:102FD000024003926246014001920091039A0B491C
:102FE00004A806F0AFF904A800F05CFF2800FFF782
:102FF00085FE0500ADE7C046FC0600205AA900008A
:103000000007002000C0FEFF04A9000046A9000040
:1030100070B50020FFF70CFE04000120FFF708FE4A
:10302000844200DA04000A4B1D686A4255412800B8
:103030001D60FFF7EDFDA0226B4252021340054ACE
:1030400028009B18044A611C1360FFF715FE70BD31
:10305000FC0600200480010000070020F8B50020D5
:10306000FFF7E6FD07000120FFF7E2FD3E00204DDF
:103070000643204C0DD18021C020C9024002FFF739
:10308000ADFD01213000FFF7F7FD1B4B2E602360E3
:103090001DE0874209DD0023B0212B60164B890219
:1030A000236023680020012517E0012380212B6085
:1030B000124BC9022360F4E7120E522A08D00028EE
:1030C00000D023600E4800F0EDFEFFF7A1FFF8BD31
:1030D00028005A68023292009B188B4205D21A6867
:1030E000561CE9D10028F2D0D1E72160EFE7C046B5
:1030F000FC060020000700200480010004C002003C
:103100001FA90000F0B585B0039203220333DC173A
:10311000294D1440E4182B68284F5A42534180220D
:103120005B42D202A4103B409B18A21C0291244E89
:10313000910000910190316800980A18934215D2CD
:10314000FFF71AFE2B685A42534180225B421F4010
:10315000D202BF183368009A9B189F4206D21948C2
:1031600000F0A0FE0025280005B0F0BD029B3568E8
:1031700019066B461A7BA423DB051343FF222F009D
:10318000090C1943019B12041B0413401943280026
:10319000FFF760FD0837281D21003760FFF75AFD53
:1031A000002C04D00A9A21003800FFF779FD009B1B
:1031B000083BFF183760D6E7FC06002000C0FEFF82
:1031C00000070020C3A8000010B5FFF7D5FD10BD13
:1031D00070B59AB0FFF742FFFF22254CD2000021C4
:1031E000200005F0D4FC0020FEF722FF04280ED1B9
:1031F0000020FEF731FF042809D1FFF709FF1D4821
:1032000000F050FE1C4800F04DFE1AB070BDFFF7F4
:103210009FFDFF25002600280ED10200C300E358C1
:103220000130591E8B41D218FF28F7D1134901A84C
:1032300006F088F801A8E3E703681A142A400A2A6E
:103240000AD11A122A40FF2A03D0D200A1180B710A
:10325000A050FFF753FDDEE7132AFAD11B122B40D3
:10326000FF2BF6D0DB00E2181671E650F1E7C046FE
:10327000701B00208FA900009FA90000A7A90000D3
:103280000021094B094A59600131516059680029F0
:10329000FCD000211961012393600222044B81318B
:1032A000FF315A501A607047FC1000400010004077
:1032B00000E100E00222064B0121DA670022054B03
:1032C0005A61054A11615A69002AFCD07047C0460C
:1032D00004E100E0FC1000400010004010B5044C78
:1032E0002378002B01D0FFF7E5FF0020207010BDF0
:1032F000050800200120024B1B685B001843704743
:103300008808002003480368002B02D114220371AF
:1033100002607047202500200120024B1B685B00E3
:10332000184370470C00002070B504000D00160013
:10333000FEF7B8FD8023012200215B055B6E627001
:10334000E270020AA271020CE2711A0A60716372E1
:10335000000EA2721A0C1B0E26702571A17020722D
:10336000E272237370BD0000124B10B51B68124C43
:103370005A1C0FD0114C002B0CD0114C012B09D032
:10338000104C022B06D00D4C042B03D00E4C052BF9
:1033900000D10B4C21000D4805F0FEFF200006F087
:1033A00003F80300042204339B0809481B0113435C
:1033B000036010BD100000203BAA000034AA0000EA
:1033C00046AA00004BAA000040AA00000C250020DD
:1033D0000825002070B5214C2278002A3DD1204BD1
:1033E00001215A608022D20511605A68002AFCD05F
:1033F000002207201B4B1C4901255A500439585004
:1034000008315A5019481A4958501A491A485A50FE
:103410001A495A50A622D2009D50082218495A50E3
:10342000043158500220174958501749174858502E
:10343000174804395850182016495850C12189009E
:103440005A500539FF395858921802435A501249B8
:10345000124A9950FFF714FF257070BD050800202F
:10346000FC000040001000400C050000746962750B
:103470001C05000024050000200004022C050000AB
:1034800014050000340500003C050000FFFF0000AB
:10349000211001005405000006080020040500006A
:1034A00070B50E4B06001B78002B01D1FFF792FF81
:1034B00000200B4D2C7884420ED00A4B2022197824
:1034C0000323091B1940084B4901C918300005F0B6
:1034D00055FB0120013C2C7070BDC0460508002042
:1034E0008C0800200408002006080020002330B5C6
:1034F00089B0984225DD03240D682C409C4220D1E0
:103500002300042D1DD90F212A681140062918D146
:1035100012091F2A15D96846FFF7C2FF23000028A9
:103520000FD06B46012218781300A04203DB6B46D4
:103530001B5D5B0013430134A1006B50202CF3D1C1
:103540000423180009B030BD70B5414B8AB01B7818
:10355000002B01D1FFF73EFF02AD2800FFF7A0FFCF
:10356000002802D100200AB070BD2B780B2BF9D9AE
:103570006B78012BF6D1EB78012BF3D10023354E7C
:10358000354C336023712B79344A1360002B0ED1F4
:10359000152169444A780B7812021A438B781B0470
:1035A0001A43CB781B0613433360002318E0012B2A
:1035B00020D1152169444A780B7812021A438B787E
:1035C0001B041A43CB781A211B06134333600E23C6
:1035D0006A7C6944934200DD130000229A4232D192
:1035E00004200021E21804339B101B0103431171D6
:1035F0002360B8E7022B03D16A7B10331621E8E77A
:10360000042B0DD1152108226944684605F0B6FA4D
:103610000098019902F08AF905F054F93060C4E786
:10362000052BC2D1152108226944684605F0A6FA87
:103630000098019902F07AF905F044F930606A7D4A
:103640000A231E21C5E78D5CA01805710132C5E76C
:1036500005080020880800202025002010000020F8
:1036600010B5134B04001B78002B01D1FFF7B2FEFD
:10367000FFF720FE00200F4A0F49104B54505860AE
:103680000130106058680028FCD00020186101301B
:10369000906018690028FCD0094B0A481B785B0130
:1036A0001B185350FFF706FEFFF7EAFD10BDC0469A
:1036B000050800200010004004050000FC10004038
:1036C000040800200608002030B589B000281EDD5F
:1036D00003230A6813401AD1042A18D90F2011684D
:1036E0000840062813D109091F2910D901240133E4
:1036F000990051580020214201D04910C8B26D46AE
:10370000591E6854202BF2D16846FFF7A9FF00200C
:1037100009B030BD10B5002813DD0C68E30710D5E3
:103720006410532C0DD8084B1B78002B01D1FFF7E8
:1037300051FEFFF7BFFDA123044ADB00D450FFF781
:103740009FFD002010BDC04605080020001000406D
:1037500010B500280EDD0C68E3070BD56410FF2CB4
:1037600008D8054B1B78002B01D1FFF733FE034A25
:10377000034BD450002010BD05080020001000406D
:103780002405000013B5002814DD0C68E30711D5EB
:10379000094B64100093094B0193072C0AD8084B7E
:1037A0001B78002B01D1FFF715FE6B46054A195710
:1037B000054BD150002016BDE2ECF0F4F8FC0004FB
:1037C00005080020001000400C05000070B588B00E
:1037D000002820DD0324086804401CD104281AD9DD
:1037E0000F2302681340042B15D1FEF741FD06009C
:1037F00005F0DAFD0500122800D912252A00022161
:103800000D326846FFF790FD6B465D73A54205DCFF
:103810006846FFF725FF002008B070BD2300325D29
:103820006B449A730134F1E7F0B50D008BB00128B9
:1038300031DD0324086804402DD104282BD90F233F
:1038400002681340042B26D14B68DB0723D5FEF713
:103850000FFD6E6807007310019305F0A5FD0500CC
:103860000E2800D90E252A000121113202A8FFF7E7
:103870005BFD6A46127902AB5A7302AA7312937304
:10388000019B76141B0ED67313745574A54205DC88
:1038900002A8FFF7E5FE00200BB0F0BD3A5D02A9DB
:1038A00063189A740134F1E730B589B0002814DD4B
:1038B0000C68E30711D5102268460021FFF734FD9C
:1038C0006B466A4665105D73684663122D0E64147C
:1038D0009373D4731574FFF7C3FE002009B030BD95
:1038E000174B184A5968002903D00021596001314B
:1038F0009160196900291FD0002018618023DB0026
:10390000D3581149012B18D1A923DB00D3585B42AE
:103910000B600E490B78032B01D801330B70032089
:103920000B490B78013303400B700A495B015B18AC
:10393000094953500123936070470860FAE7C04675
:10394000FC100040001000400C0000208C080020FB
:1039500004080020060800200405000010B5034AF2
:103960000E21034800F0B4F810BDC046C4A9000001
:10397000BBA90000044A05491368C85401339B05DC
:103980009B0D13607047C046A80C0020A8080020BB
:1039900070B5114C114A2368834202DC0023236076
:1039A00016E0155C411C2E00FA3E012E05D8994206
:1039B0000FDA555C013D1F2D01D90800ECE701002D
:1039C000151A565C6E5401318B42FADC181A2060CD
:1039D00070BD1570FAE7C046B4100020B40C00208A
:1039E00010B5FEF755FA064B1A68824201D900223B
:1039F0001A601B68C31A034898428041404210BDB8
:103A0000A4080020204E000010B5094C094A236884
:103A10001268934200D110BD074AD05CFEF772FBDA
:103A20000028F8D0236801339B059B0D2360ECE749
:103A3000AC0C0020A80C0020A808002010B5040041
:103A4000064B074A1B6812689B1ADB439B059B0DBC
:103A5000A34200DB10BDFFF7D7FFF1E7A80C002061
:103A6000AC0C0020F7B5050056680191B000441C6D
:103A700006301700FFF7E2FFFB20FFF77BFF1C205B
:103A8000FFF778FFE8B2FFF775FFE0B22412FFF707
:103A900071FFE0B2FFF76EFF6B461879FFF76AFF20
:103AA0000025AE4200DCF7BDAB00FB189C68013579
:103AB000E0B2FFF75FFF2012C0B2FFF75BFF2014F8
:103AC000C0B2FFF757FF200EFFF754FFE9E70000F1
:103AD00070B5074E3368092B08DC0C255D43054C97
:103AE0000133285164196160A260336070BDC04623
:103AF000B00C002044250020F0B587B002900C00E7
:103B0000012803DC1B20FCF7E5FC45E0244B08689A
:103B10000093830709D1042807D90F2302681340B3
:103B2000042B02D1FEF7A4FB00901D4B60680193AB
:103B3000830709D1042807D90F2302681340042BF7
:103B400002D1FEF795FB01900027164B1B680493EA
:103B5000049BBB42D6DD0C267E43134B0099F6181E
:103B6000306805F00FFC051E05D17368B668059333
:103B7000059B9D4201DB0137EAE730680199039616
:103B800005F000FC0836002808D121000298039BAC
:103B9000083102385B68984707B0F0BD0135E7E7A8
:103BA0001EA40000B00C00204425002010B5FFF733
:103BB00009F8FEF767FAFEF7BBFBFEF7F1FBFFF72C
:103BC000CDFE00F0F9FD00F07FFF10BD962210B58C
:103BD00012010021034804F0DAFF0022024B1A60B0
:103BE00010BDC04610120020AC050020064B074A4D
:103BF0001B6812689B1ADB439B059B0D01228342C5
:103C000000DC002210007047A80C0020AC0C002043
:103C1000F8B505000C0016001F1E0ED10320FFF79B
:103C2000E5FF002808D0FA20FFF7A4FEE8B2FFF76E
:103C3000A1FEE0B2FFF79EFEF8BD501DFFF7D6FFD4
:103C40000028F9D0FB20FFF795FEE8B2FFF792FEBF
:103C5000E0B2FFF78FFEF0B2FFF78CFE3012C0B279
:103C6000FFF788FE3C00E31B9E42E5DD2078FFF76E
:103C700081FE0134F7E7000070B50024F0250B4BFE
:103C80001B68A34202DCFFF7A1FF70BD2B0063435A
:103C9000074A9B181A78002A05D05978002311206A
:103CA0001A00FFF7B5FF0134E9E7C046AC05002074
:103CB00010120020F8B507000024F0252B00634304
:103CC0000C4A01349E18B74211D0317800290BD02C
:103CD0000133D15C002311201A00FFF799FF2A005D
:103CE0000021300004F053FF0A2CE7D1F8BD024B4D
:103CF0001C60F9E710120020AC050020F3B50400A9
:103D0000100001220300FFB00D00134013D002ABDE
:103D10001A70431002AA02A9537042121B0E8A7035
:103D20000B7105220B004014C87029002000FFF71A
:103D30006FFF7FB0F3BD032606401ED104281CD9B7
:103D40000F2201680A40042A29D1022302AA137013
:103D5000FEF78EFA070005F027FBF823FF339842A1
:103D600000D91800B04202DC421C02ABDDE701368C
:103D7000731EFB5C02AA9355F4E7042801D00028C7
:103D800009D1032302AA043813704242504102AB06
:103D900058700222C9E7002ECBD10428C9D90F21BF
:103DA00002681140052913D1013902AE3170F821A2
:103DB0001209FF3192008A4200DD0A00934201DBC2
:103DC0000132D2E70133C118C97802AEF154F5E7E8
:103DD0000629AED101390E00120956430196F82684
:103DE000019FFF36B742A4DC02AE31700136934228
:103DF00001DB019AE4E70127013399004158394278
:103E00000BD03941012737700F127170B7700F1442
:103E1000090EF77031710536E9E70149F2E7C0464E
:103E200019FCFFFF70B502000024F0210D4E0800C0
:103E3000604380194578954203D001340A2CF6D1AD
:103E400070BDF022002104F0A2FE074A1368013B76
:103E5000A34200D11460002329001A001120FFF7AB
:103E6000D7FEEDE710120020AC05002010B5B2B06F
:103E700002236A460400137005F096FAC72800D999
:103E8000C7200023984207DC421C6B46FE21142009
:103E9000FFF7BEFE32B010BD694601335A1EA25C68
:103EA000CA54EFE730B5B3B002236A460500137079
:103EB00005F07AFA0400C72800D9C72400239C42E1
:103EC0000BDC20003230FFF7B9FD621C6B46FF218E
:103ED0001420FFF79DFE33B030BD694601335A1EF2
:103EE000AA5CCA54EBE70000F7B5234B06001B6839
:103EF000F02100930023009A9A4211DC0024F02361
:103F00001A006243019201991C4A55182F78002F1C
:103F100012D001340A2CF3D11948FFF7C3FF29E06E
:103F20000A005A43154882185078B04202D11278DC
:103F3000002A1FD10133DEE7F0223900280004F007
:103F400026FE02230D4A0199EB6053540D4AF100FD
:103F50008A58009B6E70AE70AA602F616F61A34299
:103F600002DC054B01341C60002331001A001020D4
:103F7000FFF74EFEF7BDC046AC0500201012002032
:103F800035AF0000701B002010B5FFF775FEFF2451
:103F9000084AE3005B429B18074AD35C043B012BB1
:103FA00003D8E043C0B2FFF79FFF013C002CEFD1E4
:103FB00010BDC046FC070000701B0020F7B50E00C6
:103FC000FF247F2501901C4AE300D31A1B4A9A184C
:103FD0001278062A01D0032A1DD1FF22D2009B1895
:103FE000186883682B401C2B15D1C3681A002A401F
:103FF000042A10D102692A40192A0CD11B0A013364
:104000009B000C30C018FEF733F9070005F0CCF91F
:104010000023B04209D0013C002CD4D1F7BD019A55
:10402000F95CD25C9142F6D101339E42F7DCE04369
:10403000C0B2FFF759FFEEE7701B0020FC0700003D
:1040400070B50500FF24084AE3005B429B18074A4D
:10405000D35CAB4203D1E043C0B2FFF745FF013C64
:10406000002CF0D170BDC046FC070000701B002082
:10407000F7B5FDF70DFF514B1A68824201D90022B6
:104080001A601A684E49821A8A4200D883E0186082
:10409000FDF708FF071E00D101370020FDF7C8FF1C
:1040A00001900020FDF7D8FF019B0090454C464D44
:1040B000002B14D02368002B00D07AE02B682760F7
:1040C000002B00D171E0414B01261B78002B63D1FE
:1040D0000920FFF7B5FF3E4B1E703C4B1E70009B46
:1040E000002B12D02B68002B0FD123682F60002BE0
:1040F0001ED0374B01261B78002B52D10920FFF729
:104100009FFF334B1E70314B1E702368002B0FD066
:104110002F4E3278002A0BD19F4200D227602368AD
:10412000FB1A312B04D90720FFF78AFF01233370D4
:104130002B68002B0FD0254E3278002A0BD1BB42C2
:1041400000D92F602B68FF1A312F04D90820FFF700
:1041500077FF012333702368002B0CD0019B002BC9
:1041600009D11B4E3378002B02D10720FFF768FFDF
:104170000023236033702B68002B0CD0009B002B96
:1041800009D1124C2378002B02D10820FFF758FFE9
:1041900000232B602370F7BD0720FFF751FF0C4B66
:1041A0009CE70820FFF74CFFADE7009B002B9CD15C
:1041B000ABE7009A002A95D1AAE7C046A0080020E4
:1041C0000F27000090080020980800209C0800207D
:1041D0009408002037B500240500FFF74DFD01A825
:1041E0000194FDF713FF21002000FEF7D5F9FEF73B
:1041F00093FBFDF745FFFDF744FFFEF7D9FCFDF704
:104200006DFEA54204D0FDF793FF0248FFF74AFE7A
:1042100037BDC04626AF0000002310B501001A00CC
:104220001120FFF7F5FC10BD07B56B461970694604
:104230005A7013128B701314120ECB700A716B46E6
:10424000010005221320FFF7E3FC07BD10B50A00AB
:1042500001001220FFF752FD10BD70B505000800E7
:104260000C003230FFF7EAFB2B00220000211B205C
:10427000FFF7CEFC70BD10B50C0003001100142038
:104280002200FFF7C5FC10BD012370B5FF24084ACA
:1042900041185B42884201D3D84370BD06781D0A9D
:1042A000234073409B009B5801306B40F2E7C046AF
:1042B00008AB0000002313B501930B4BC2000400B0
:1042C000D058002805D0436808309900FFF7DCFF7C
:1042D00001900920FFF7B2FB01AB04222100172057
:1042E000FFF796FC13BDC046701B002070B506009A
:1042F0000020FEF703FD0024FF25002801D1200047
:1043000070BD03681A142A40152A07D11B122B40CE
:10431000B34200D10400FEF7F1FCEEE71D2AFAD10A
:104320000024F8E7F0B580279DB0FFF76DFBAD4C9A
:10433000AD4D2068FF00391A4019FDF7C9FE23680A
:104340000600C3182360002B0ED11DB0F0BD2068FD
:10435000391A2818FDF7BCFE236806001B182360D5
:10436000FDF796FDA14B1860002EF0DC2B78FA2BA0
:1043700000D013E12368022B07DCFFF731FB002894
:10438000E3D00120FFF704FBDFE76878AC78023860
:1043900018281FD802F046FD0D2024282B341E3E7D
:1043A0006872768CDEEF1E1E1E1E1E1E1E1E1E1E38
:1043B000FD00FF2C0ED02000FFF734FD00228C4BB7
:1043C000E100CA505B181A712100009213001320FB
:1043D000FEF798FE0320D5E72000FFF785FDF9E7FB
:1043E0002000FFF71FFDF5E7FFF7CEFDF2E7FFF72F
:1043F00043FC0020FFF7EEFE7E48FFF753FDE9E7A0
:10440000632CE7D87C4BA200D25821001520FFF77F
:1044100075FCDFE700242000FFF768FF061E03D1CC
:104420000134642CF7D1D5E7083004F0BDFF050056
:104430000530FFF703FBFB20FFF79CFA1D20FFF779
:1044400099FAE0B2FFF796FAE8B2FFF793FA28126A
:10445000C0B2FFF78FFA3700BB1B9D42E0DD387A10
:10446000FFF788FA0137F7E700211D2000910B00C4
:104470000A00FEF747FEFDF75BFEABE72000FFF703
:1044800019FFA7E7FDF716FD03AC5C4A6421009015
:104490005B4B200004F024FF02232000237004F073
:1044A00083FF2300020000211620FFF7B1FB91E7F4
:1044B00000244F4AE300D558002D28D06B689E0099
:1044C000701DFFF7BBFA2B000025320008332100D6
:1044D0000120FFF79DFB0020FEF710FC2F002E00AF
:1044E000002818D1002F04D03A0001212000FFF746
:1044F000B9FA002D04D02A0002212000FFF7B2FAF9
:10450000002E04D0320000212000FFF7ABFA013466
:10451000FF2CCED15EE7FF2103681A120A40A242A7
:1045200009D11A140A400B2A08D10B400CD0012BD8
:104530000CD0022B0CD0FEF7E1FBD1E7132AFAD105
:1045400000252F002E00F6E70600F4E70700F2E74B
:104550000500F0E70024FFF78FFB22002100009404
:104560002300DA20FEF7CEFDFF222100D2002048F2
:1045700004F00DFB7FE7012C02D1FEF7E1FC29E7F7
:10458000022C02D1FEF720FE24E70120FFF722FED5
:1045900020E7002321001A001A2086E7FB2B00D019
:1045A000EFE62268042A00DCE7E62E79E878154B6E
:1045B000360206439E4200DDE3E6331D9A4200DCEC
:1045C000DBE6EB5CFE2B00D0DBE66B78AC78711E93
:1045D0001B2B6BD018D8012B2BD0082B3DD0701D76
:1045E000D0E6C046B4100020B40C0020A40800207F
:1045F000701B002008AF0000682300201FAF0000E0
:104600001AAF0000F60300001D2B60D052D31E2B02
:10461000E5D1012CE3D10029E1DD6B79002B03D03A
:104620001C00322B00DD322464235C43344B1C60BD
:10463000D5E7FF2CD3D02000FFF7F4FB6D79314A8A
:10464000B31E009221002A000A20FEF75BFD2E4BCC
:10465000E400E0501B191D71C1E7632CBFD86A79D3
:10466000022A13D0032A1BD0012AB8D1E979AB79E9
:10467000090219432B7AA4001B0419436B7A1B0609
:104680000B435B001343214AA350A8E70029A6DD92
:10469000B11E1C48FDF7D0FD1C4BA400E0509EE766
:1046A000AB79A4005A1E93419B00ECE71848FFF732
:1046B00085FC94E7FF2C92D06A79022A8FD81149A1
:1046C0000B2000912100B31EFEF71CFD87E70B00B5
:1046D000632900DD6323002203A893420ADCD94347
:1046E0000022C917194041180A70013300902100B7
:1046F0001520E9E7A918497981540132EDE7C04650
:1047000004000020BA0C0020701B00206823002049
:10471000B90C00200120704710B5064C200000F0B5
:104720000BFB0549200000F02FFB0122034B1A6010
:1047300010BDC046E0100020801A0600B81000200E
:1047400010B501210D20FDF7BBFB01210E20FDF767
:10475000B7FB00210F20FDF7B3FB044C200000F055
:1047600027FA1021200000F03FFA10BDC0100020F1
:1047700010B504680D20E30703D56410FF2C03D99E
:104780001720FBF7A7FE10BDFFF7DAFFE1B20248E2
:1047900000F04CFA0020F6E7C010002010B5FFF73B
:1047A000CFFF0021034800F041FA430001201843E5
:1047B00010BDC046C010002010B5034A07210348B1
:1047C000FFF786F910BDC0464CAF000084AF000073
:1047D000F8B5012306681E4205D045681D4202D087
:1047E00084681C4203D10D20FBF774FEF8BD7610DF
:1047F0001520802EF8D86D101620FF2DF4D86410E7
:10480000FF2C01D91720EFE70B4B1B68002B01D1C0
:10481000FFF782FF094FF1B2380000F04CFBE9B21C
:10482000380000F04FFAE1B2380000F04BFA3800DF
:1048300000F0ACFB0020D9E7B8100020E010002009
:10484000F7B501242300A0421BDD0D682C4218D0CF
:104850001A4B25411B684C68002B01D1FFF75CFF08
:104860000127174EE9B2300000F025FB3C420AD088
:104870003C413000E1B200F025FA300000F086FB48
:1048800000231800FEBD03252540F6D1042CF4D9E1
:104890000F2322681340062BEFD113090193019BCC
:1048A0009D42EADA0135AB00E1583942F7D04910B0
:1048B000C9B2300000F006FAF1E7C046B810002097
:1048C000E0100020144B70B51B6805000E00002B93
:1048D00001D1FFF721FF114CEDB22900200000F0BB
:1048E000EAFAF1B2200000F0EDF90021200000F01A
:1048F000EDFA002801D0404270BD012229002000BD
:1049000000F0D4FA200000F0CEF90028FAD0200000
:1049100000F0CEF9F0E7C046B8100020E01000200B
:1049200010B501240368234202D04168214203D11B
:104930000D20FBF7CFFD10BD5810802801D91520A0
:10494000F7E74910FF2901D91620F2E7FFF7BAFF70
:1049500040002043EFE710B507211820FFF7B2FF12
:104960007F2801DD0138FF3803007F3301DA7F2023
:10497000404264235B4258437F2102F0E7FA01235F
:1049800040424000184310BD10B508211820FFF721
:1049900099FF0300C00FC0180123401015304000DC
:1049A000184310BD10B505211820FFF78BFF7F2895
:1049B00001DD0138FF3803007F3301DA7F204042F8
:1049C00064235B4258437F2102F0C0FA4300012078
:1049D000184310BD10B503211820FFF773FF7F287F
:1049E00001DD0138FF3803007F3301DA7F204042C8
:1049F00064235B4258437F2102F0A8FA4300012060
:104A0000184310BDF8B50123020018009A4236DDA4
:104A10000E68334233D003244D682C402FD1042D2F
:104A20002DD90F2229680A40062A28D1144B1B6869
:104A3000002B01D1FFF770FEEB0704D42B681C0993
:104A4000202C00DD20247610F1B20E4E2200300022
:104A500000F02CFA0435A700EF19AF420CD030005B
:104A600000F021F90028FAD0300000F021F90123EC
:104A70004000184301C5F0E7012064002043F8BD61
:104A8000B8100020E010002000207047012070477F
:104A900000207047002070470120704700207047B9
:104AA00000207047002070470020704700207047AA
:104AB000002070470020704700207047002070479A
:104AC000704770477047000010B5034A0E21034835
:104AD000FEF7FEFF10BDC046C8AF000038B00000B2
:104AE00010B5FDF7DBFA0648FDF746FBFFF75EF869
:104AF0000448FFF7D7F9FEF76BFBFFF745FA10BD47
:104B0000E2040000C1B0000010B5FDF75BF910BD74
:104B100070B5002504AC24780573A94205D10A4B71
:104B20000A4A23210A4803F0ADFF016009499200B7
:104B300052589B0002715B58A400837163588560D2
:104B400043710223C37170BDD9B000003EB10000B3
:104B5000E7B000009CB10000037B002B04D143733D
:104B60008373036101330373704700001FB5019124
:104B7000A02100240068C900D2B24450012A10D0FC
:104B8000A24209D0032A0AD0074A8350074B019A50
:104B9000C250012343501FBD02221343F4E70422F5
:104BA000FBE70622F9E7C046540500002405000093
:104BB00010B50400FFF7D0FFA1222368A179D2002D
:104BC00099506179064A2000995021790432995010
:104BD000044B19685A689B68FFF7C8FF10BDC046B0
:104BE0000C050000D41000204BB2002B0FDB8023FB
:104BF0003F290FD81F290FD80F290FD807290FD801
:104C000003290FD81B060168074A8B507047802381
:104C10009B04F8E7DB04F6E71B05F4E75B05F2E726
:104C20009B05F0E7DB05EEE7240500000368074A73
:104C300099501A00FC32D1680029FCD0A321C90088
:104C400058580023C0B2D3607047C0461C0500000E
:104C500007B58022074BD2051A6000229A60023203
:104C60001A7111230E320093034905330348FFF7ED
:104C70004FFF07BDD410002000300040C0100020BE
:104C8000F8B505000E0017000024BC4208D02B68C0
:104C9000315D1B6828009847002801D00134F4E7F3
:104CA0002000F8BD704710B51C3000F0A9F910BD08
:104CB00010B51C3000F096F910BD10B51C3000F096
:104CC000A5F910BD70B5437E0D00002B01D1002069
:104CD00070BD6430040000F0A2F90028F7D1200074
:104CE000290000F070F90120F2E70000F7B5019308
:104CF000FA23002504009B0083600D4B45600833B8
:104D000003601C300F00160000F052F920006430E0
:104D100000F04EF9074A2761B600B35820006375CA
:104D2000019B9B009B586576A576A375FEBDC0468A
:104D30007CB100009CB100000123A022C375837DDB
:104D40000E49C133FF33D2059B009950437DC133D7
:104D5000FF339B009950CC220169094B5204CA5081
:104D600005220169243BCA50827D01690833CA507B
:104D70000269417D034BD1507047C0460C060000CC
:104D8000240500000C050000A022002310B50469D2
:104D9000D200A3500A4CA1420FD90A4C8C425B416D
:104DA00009495B420B40CD21C9045B1804690749DE
:104DB000635005210369995010BDCC235B04F5E7CE
:104DC000A086010090D00300000098FD240500009B
:104DD000F7B5040000200D000193824265D0160053
:104DE000402A00D9402627001C37380000F0F6F88A
:104DF000B1232269DB00D550802201232169920072
:104E00008B50A27E002A03D12269136222691360AB
:104E10000025731EAB4207D1019B002B04D08022DA
:104E20000221236992009950012223691A622369A1
:104E3000FC33DA68002A02D19A6A002AF9D09A6A09
:104E4000002A0BD1DA60A3232269DB00D158380095
:104E5000C9B2013500F0B7F8B542DAD3019B226937
:104E6000002B0FD11300FC339B6A002B0AD10133B6
:104E7000A376D3612369FC33DA6C002AFCD00022CC
:104E8000DA640AE000230121A37651611A00236944
:104E9000FC3399680029FCD09A602369FC339A6A34
:104EA000002A01D000229A62E8B2FEBD10B50123AB
:104EB000FFF78EFF10BD0300AC3310B5040019706E
:104EC000643000F08BF80123637610BD00230200EC
:104ED00070B5AC3243760D001178B1220400006940
:104EE000D20081508022216992008B5022690133C7
:104EF00013622269936026006436300000F080F867
:104F0000002812D0300000F06DF81E4B2269D050FE
:104F10002369FC331A6A002A02D19A6A002AF9D05E
:104F20009A6A002A01D11A62E5E723690122002D5D
:104F30000DD11900FC31896A002908D1DA61236991
:104F4000FC33DA6C002AFCD00022DA6407E05A61F4
:104F50002369FC339A68002AFCD000229A60002062
:104F60002369FC339A6A82420BD098622169064A0F
:104F70008B588B501800022B03D0181F431E9841EA
:104F8000033070BD1C050000C404000010B50121F1
:104F9000FFF79CFF10BD000010B513231222024939
:104FA0000248FFF7A3FE10BD00400040E0100020C3
:104FB00010B540220021040003F0E9FD0023200089
:104FC0002364636410BD10B53F24026C531C23405E
:104FD000446C9C4201D08154036410BD00230364DF
:104FE00043647047436C026C934206D03F21C25C1D
:104FF00001330B4043641000704701204042FBE73F
:10500000036C406C181A00D540307047436C026C3A
:10501000934201D0C05C704701204042FBE73F2231
:10502000036C406C01331340181A43425841C0B21C
:105030007047000003210A4802680A4302600948D9
:1050400002680A4302600849084A094B9B1A03DDBB
:10505000043BC858D050FBDC00F012F8FBF754F8C2
:1050600024050040540500409CB6000000000020CC
:1050700044020020FEE7FEE7FEE7FEE7FEE7FEE76C
:105080002D4B10B51A68D2B2012A0FD12B4A1268E3
:1050900012070BD12A4AE0241168F02208001040C0
:1050A00021422DD12749096811422CD01A68D2B269
:1050B000012A12D12149096809070ED1F02020499F
:1050C00009680140402908D11E490968014204D1FC
:1050D0008020C121C005C90042501B68DBB2012BF2
:1050E0000DD1164B1B681B0709D1154B1A68F0230D
:1050F0001A40A02A0FD1134A12681A420ED010BDCE
:105100003028CFD0D2E7104A104911608021104AD0
:1051100009021160CAE7D02AF1D1ECE70D4B1A68F9
:10512000012A04D00C4A1A601A68012AFCD1C02254
:105130000A4B1A60E3E7C046E00F00F0E40F00F00E
:10514000E80F00F0EC0F00F004050040DFFF07C09F
:10515000186C004000EC06407593000014EC06400B
:105160000120704710B503681322DB69984710BD12
:1051700070470000054B0269D1500369FC331A6A7D
:10518000002AFCD0002201201A6270471C05000092
:10519000030010B55C331A781F231A401E3B190018
:1051A0009140114AD167C222042104699200A150A2
:1051B000026953600269D360A02300220169DB0009
:1051C000CA5001230169094A5B428B500169084AB0
:1051D0008B5001690C3A8B50016908328B501430A6
:1051E000FFF7FCFE10BDC04604E100E00C05000026
:1051F0001405000010B51430FFF702FF10BD10B504
:105200001430FFF703FF10BD10B51430FFF7EAFEAE
:1052100010BD0000030070B55E331A780469724B4C
:10522000E25003005D331A780469704BE2500300CA
:1052300061331C7802696E4B012C00D09EE00500A2
:105240005F352E78A225ED005651020060321578A8
:10525000A1220669D200B5500269D4509623DB0022
:10526000994200D88CE096231B01994200D88AE02D
:1052700096235B01994200D888E096239B019942CE
:1052800000D885E0E1239B01994200D882E0962373
:10529000DB01994200D880E0E123DB01994200D88C
:1052A0007DE096231B02994200D87AE0E1231B029D
:1052B000994200D877E096235B02994200D874E0C7
:1052C000E1235B02994200D871E0E1239B029942FD
:1052D00000D86EE0474B994200D86CE0E123DB0236
:1052E000994200D86AE0E122002312038A425B411E
:1052F000414A5B421340802252059B1801693F4A94
:105300008B50A02304220169DB00CA5000210369ED
:10531000FC33D9600369FC331962012301690B6016
:1053200001698B60C1210469890062501F215C30D2
:1053300002780A4093406231314AFF3153500021D4
:10534000415600293CDA0F230B40083B2D4C9B08AB
:105350009B001B1903242140A140FC348C40DD69D3
:10536000A5432C00C0258D4029002143D9611F236E
:10537000017819401E3B8B40136070BD00246CE720
:105380009E23DB02BAE79D231B03B7E71E4BB5E75D
:105390001E4BB3E7EC239B03B0E71D4BAEE71D4B61
:1053A000ACE71D4BAAE71D4BA8E71D4BA6E71D4B1D
:1053B000A4E71D4BA2E78023DB049FE71B4B9DE77F
:1053C0008C080F4BA400E41803230B40FF21C025D9
:1053D000DB009940AD0066598E433100C0269E40E7
:1053E00033000B436351C2E70C05000014050000B5
:1053F0006C05000090D0030000D0BEFE2405000024
:1054000000E100E000ED00E000B0130000502700D4
:1054100000A04E0000F0750000509D0000F0EB0071
:1054200000903A0100E0D70100B0AF0300705F07C1
:10543000F7B5009308AB1B7800250193FA2304000D
:105440009B0083600E4B45600833036014300F00EF
:105450001600FFF7ADFD23005C3327611E70009B33
:10546000084A9B00995823005D331970019B200066
:105470009B009A5823005E33DD701A70FEBDC04653
:1054800018B200009CB10000036910B51A00FC328C
:10549000D2680400002A0AD0A322D20099581430FE
:1054A000C9B2FFF790FD00222369FC33DA6010BD1A
:1054B00010B50248FFF7E8FF10BDC0469811002064
:1054C0001D2307B502220093024901330248FFF76A
:1054D000AFFF07BD0020004098110020704700007A
:1054E00010B500F011F8FFF7F9FF012000F000FA05
:1054F000FFF7F6FAFFF708FB024B002BFAD000E0AB
:1055000000BFF7E700000000C420114B80001A58CC
:1055100010491140C02212020A431A50C0218022B1
:10552000490092025A501A608023A3220021DB0511
:10553000D20099500122F9309A60074BFF30195080
:10554000C120023180001950403019501A60704754
:1055500000E100E0FF00FFFF00100140014B186078
:105560007047C0465C000020F7B500231E285AD8BB
:10557000384B8000C258042A5BD007D8022A54D086
:1055800055D80423012A09D000234CE0062A54D020
:1055900051D31A2A53D002231B2AF5D12E4A11685F
:1055A00008294ED909294FD00A240226A020012516
:1055B0002A4AC00015502A482A4D07681C20BF00FF
:1055C00007402948019700685759009027481B0257
:1055D00007401F43C02300989B020340FF20575100
:1055E0005759000207401F43019B1F43009B58016E
:1055F0006023184007433E43565101251C4B15605C
:1056000058680028FCD000205860A1230125DB0049
:10561000D3585560A025ED0050511BB2A14202D0D5
:1056200015D2611ACB401800FEBD0823B6E710233F
:10563000B4E72023B2E74023B0E78023AEE701239D
:10564000ACE708240026B1E70C000126AEE7091BF1
:105650008B40E8E79CB1000058000020007000403B
:10566000140000200405000018000020FF00FFFFC8
:10567000FC700040F0B51E285BD8364B8000C25845
:10568000354B1E68002E30D1C227344BBF00D8598D
:10569000334C03250440C02000022043D851C024CD
:1056A00080206400800018512E4F18602E4B803CE3
:1056B000D859FF3CA043D8510437D859A8432043B8
:1056C000D8510837D8590C35A84384460720654679
:1056D0002843D851A820C0001E50C1208026800039
:1056E00076021E501C601C4B1C60142500202B00F1
:1056F0001E4C2E0046433659771C1BD14343E250C3
:10570000A0230325C132FF329200DB05D550184B90
:105710001A68082A14D114234343E3189A681248DC
:105720005132FF32920059601150DA68C1239B0058
:10573000C250F0BD9642E1D001300328D9D1F8E73C
:10574000082A02D9083AD140E5E708239A1A91407D
:10575000E1E7C0469CB10000FC11002000E100E040
:10576000FF00FFFF04050000009000401C00002027
:105770005C0000202149F0B54A6C2148002A14D071
:10578000A025A12600230124ED05F600C258571CD0
:1057900006D0C7187F68002F02D027009740AF516E
:1057A00014333C2BF2D100234B64A0230121DB05F1
:1057B00000260F009C4614234B43C3181A1F12687F
:1057C000104C0E4D920014195219526C002A10D030
:1057D0001A00143A1268551C09D0103B1B68FF2BA5
:1057E00005D03B00934065461A00074BEA50FC3455
:1057F000666401310429DED1F0BDC046FC90004052
:105800001C000020009000400C05000000B51E2880
:1058100010D80C4A8000835803290BD8A022080016
:10582000C133FF33D2059B0001F0FCFA02090507E2
:105830000021D15000BD0C21FBE70421F9E7032131
:10584000F7E7C0469CB100001E280AD8074B80002D
:10585000C25801239340A022D205002902D1044955
:1058600053507047A121C900FAE7C0469CB100001F
:105870000C050000030000201E2B0AD8A021A22244
:10588000C905D2008858034A9B009B58D840012381
:10589000184070479CB10000F7B506000D000C00E1
:1058A0008B180193019B671B9C4207D033682178BA
:1058B0001B683000984701340028F3D13800FEBD42
:1058C0000849094A094B10B51B688858FA22190A79
:1058D0001B0618439200002301F070FC4904C00B22
:1058E000084310BD00100140040500000012002014
:1058F00070B5041E09D0FFF7E3FF050000F014F8AF
:10590000FFF7DEFF401BA042F8D370BD0022044B1E
:105910009A60044A13680133DBB213607047C046D3
:10592000FC1001400012002070470000F0B5C64690
:1059300000B5CB0F9846404A4B005B0D9A1882B0D9
:105940000D000400132A2FDC002A49DB3B4F1741CE
:105950003E000E40064323D07F08390029400C4307
:105960000AD03749BD438C4663445C425C41802386
:10597000DB021341E4071D434146CE0031492B00B1
:105980008E192200346875682000290001F0BCFDE2
:10599000009001910098019922002B0002F04AFC2E
:1059A00002B004BC9046F0BD332A08DD8023DB0042
:1059B0009A42F5D102000B0001F0A6FDF0E7224A61
:1059C0009446012263445242DA400242E8D052082F
:1059D0000242D1D094438022D2051A411443CBE72E
:1059E0004B005B080343DBD00B031B0B1C436342E0
:1059F000234380244D0C24031B0B23406D042B43B5
:105A000019004346DA000F4B9B181C685D680200C2
:105A10000B002000290001F077FD00900191009813
:105A2000019922002B0002F005FC42464B005B0866
:105A3000D60733431900B3E701FCFFFFFFFF0F0058
:105A4000EEFBFFFF48B20000EDFBFFFFF8B5274A71
:105A50004B005B0D9A180C000700132A10DC002A7B
:105A600036DB234B13410B423AD0802424031441EC
:105A7000002064189C430600250030002900F8BD72
:105A8000332A0EDD80230600DB000D009A42F4D19C
:105A900002000B003800210001F036FD06000D0069
:105AA000EBE7144D0600AC46012563446D42DD4032
:105AB000AC4663460D000342DFD033239A1A323BD3
:105AC00093401818874200D94C1C63469843D2E78C
:105AD000C90FCC070020531CCDD1074B1C43CAE78C
:105AE00006000D000028C0D1C7E7C04601FCFFFF3B
:105AF000FFFF0F00EDFBFFFF0000F03F30B5214A34
:105B00004B0087B05B0893421EDD1F4A934205DDC0
:105B100002000B0002F08EFB07B030BD02AA00F0BD
:105B200035F803231840049A059B012813D0022856
:105B30001DD0002814D00298039900F037FA802372
:105B40001B069C466144E7E70023002200930023E4
:105B500000F0A6FFE0E70298039900F027FADBE7E0
:105B6000012402980399009400F09AFFD4E70124DD
:105B700002980399009400F093FF80231B069C4633
:105B80006144C9E7FB21E93FFFFFEF7FF0B54E46D7
:105B90004546DE465746E0B5E14B4C008FB0904697
:105BA000894664089C4200DC87E0DE4B9C4222DC94
:105BB000DD4A002900DC92E0DC4B02F03BFBDB4BD2
:105BC00006000F009C4200D17EE1D94AD94B02F079
:105BD00031FB02000B00414630000A604B60390087
:105BE00002F028FBD34BD24A02F024FB43460125A6
:105BF0009860D9606BE0D04B9C4200DC8FE0CF4BCB
:105C00009C4200DD55E1CE4A231592469A44514606
:105C10000905631A19001D00040002F053FE02F08A
:105C200087FE02000B00200029000892099302F071
:105C300001FB0022C34B02F08BF80F00060002F0BC
:105C400041FE02F075FE04000D0002000B00300062
:105C500039000A940B9502F0EDFA0022B94B02F0DC
:105C600077F8002200230C900D9101F079FA0028BA
:105C700000D192E1002300222000290001F070FAF7
:105C8000434243410133B04A41460192022208A8EF
:105C90000092524600F0A4FA4B460500002B16DA9B
:105CA000802243461206944642465B68454263445E
:105CB0005360D3686344D36009E00B00020041469F
:105CC0000A604B600022002300258A60CB60280018
:105CD0000FB03CBC90469946A246AB46F0BD934BF4
:105CE00001F012FC914B06000F009C4200D13DE1F7
:105CF0008F4A904B01F008FC02000B004146300037
:105D00000A604B60390002F095FA894A894B01F02C
:105D1000FBFB012543466D429860D960D7E700F050
:105D200071FF8A4A8A4B06000F0002F011F8002228
:105D3000884B01F0E9FB02F0C5FD050002F0F8FD1B
:105D4000794A7A4B0490059102F002F802000B00A8
:105D50003000390002F06EFA754A06000F00049810
:105D60000599744B01F0F4FF029003911F2D00DCA4
:105D7000C7E0029A039B3000390002F05BFA8346C9
:105D80008A4653465B0024155B0DE31A102B6CDD2D
:105D900004980599D322674B520501F0D9FF020000
:105DA0000B00300039000292039302F043FA0A001C
:105DB000010013000691079202003900300002F042
:105DC00039FA029A039B02F035FA06000F00049894
:105DD0000599614A614B01F0BBFF32003B0002F0C4
:105DE00029FA069E079F0B0002003900300002923C
:105DF000039302F01FFA4B005B0D83468A46E41AB8
:105E0000312C32DD04980599B822544B920501F0EB
:105E10009FFF03000C000200029303940B000698FE
:105E2000079902F007FA02000B0006000F0006981F
:105E3000079902F0FFF9029A039B02F0FBF9484A26
:105E40000290039104980599464B01F081FF029A54
:105E5000039B02F0EFF902000B00300039000292C0
:105E6000039302F0E7F983468A465A465346414671
:105E700030000A604B60390002F0DCF9029A039BA3
:105E800002F0D8F944460B000200A260E3604B46E2
:105E9000002B00DB1BE75B46236080231B0653447B
:105EA000636080231B069C466144A060E1606D42F4
:105EB0000DE70B00020002F0BDF943460025986093
:105EC000D9601860596002E7D3221A4B520502F0DC
:105ED000B1F9214A214B0D00040002F0ABF9020098
:105EE0000B00414620000A604B60290002F0A2F935
:105EF0001A4B194A02F09EF9434601259860D96071
:105F0000E5E602000B003000390002F093F96B1E49
:105F1000154A9B009B5883468A46A342A5D130E789
:105F2000FB21E93F7BD9024000004054FB21F93FAF
:105F30003163621A61B4D03DFB213941FFFFEF7F2D
:105F4000EAFBFFFF00007041D8B2000083C8C96DB2
:105F5000305FE43F0000E03F7370032E8A19A33BDB
:105F6000C14920259A837B3958B20000D3220C4BBB
:105F7000520501F0C9FA0B4A0B4B04000D0001F069
:105F8000C3FA02000B00414620000A604B60290062
:105F900002F050F9034A044BB9E6032373E6C04606
:105FA00061B4D03D7370032E8A19A33BF0B5474608
:105FB000CE4680B587B000920193754B4F00814665
:105FC00088467F089F4263DC02F07CFC002800D1F9
:105FD000D4E04A4643464846414601F0B9FE040033
:105FE0000D006C4A6C4B01F0B3FE6C4A6C4B01F037
:105FF0008BFA22002B0001F0ABFE6A4A6A4B02F0DA
:1060000019F922002B0001F0A3FE684A684B01F049
:106010007BFA22002B0001F09BFE664A664B02F0E1
:1060200009F922002B0001F093FE644A644B01F051
:106030006BFA22002B0001F08BFE029003910022EC
:10604000604B2000290001F083FE029A039B0600AA
:106050000F002000290001F07BFE009A019B040044
:106060000D004846414601F073FE02000B0020007F
:10607000290002F0DFF802000B003000390002F0C6
:10608000D9F802000B0000204F4902F0D3F870E06D
:1060900002000B0001F05CFE04000D003D4A3E4B87
:1060A00001F056FE3D4A3E4B01F02EFA22002B0035
:1060B00001F04EFE3B4A3C4B02F0BCF822002B00A4
:1060C00001F046FE394A3A4B01F01EFA22002B003D
:1060D00001F03EFE374A384B02F0ACF822002B00AC
:1060E00001F036FE354A364B01F00EFA2B00220045
:1060F00001F02EFE354B029003919F429FDD344B01
:1061000000229F423DDC334900207B182E491600B7
:106110001F0002F08FF8049005910022294B200007
:10612000290001F015FE32003B0002F083F8029ACC
:10613000039B06000F002000290001F009FE009AD1
:10614000019B04000D004846414601F001FE02009B
:106150000B002000290002F06DF802000B00300057
:10616000390002F067F802000B000498059902F06C
:1061700061F807B00CBC90469946F0BD002012496A
:10618000F7E7154B002604920593144FC5E7C04668
:10619000FFFF3F3ED43888BEE9FAA8BDC4B1B4BD04
:1061A0009EEE213EAD529C804F7E923E9015CB19C3
:1061B000A001FA3E7751C1166CC1563F4C5555555A
:1061C0005555A53F0000E03F0000F03F3233D33F7C
:1061D0000000E93F0000E0FF0000E73F0000D23F81
:1061E000F0B5DE464E4645465746E0B5DC4CA54484
:1061F0000D9114001900A49A0993DA4B9200D65815
:106200004D1E03901821E01E0696029500F09EFE9A
:10621000C3430100DB1719404B1C9A009B1ADB009B
:106220001B190B9105934C1B771918D4A59BA5003E
:106230009C463F1922AE6544013707E0286802F00A
:1062400077FB013403C60435BC4208D0002CF5DAD4
:1062500000200021013403C60435BC42F6D1069B60
:10626000002B01DA00F0FDFB069B03990133DB00F4
:106270009A46099BDA00944600920022914672AA3F
:106280000492B94A6144934688469AAB63449B445E
:10629000029B002B00DABCE15D4600260027039C30
:1062A0004D442A686B6803CC01F052FD02000B00DC
:1062B0003000390001F028F9083D06000F00444580
:1062C000EFD1049B4B441E605F6008239C46E14471
:1062D000D145DDD10EA804218446494261448C4653
:1062E000069A93009C44614684460A910399083BB0
:1062F00063448C460C93009B009263449B46009A37
:106300000498D10003008C46634408911E685F68BE
:10631000002A33DD954980468C466244D300984478
:1063200070AB9A460EAB99460022914B3000390073
:1063300001F00EFD02F0C6FA02F0FAFA00228D4BCF
:1063400004000D0001F004FD02000B0030003900D4
:1063500001F070FF02F0B6FA4B4601C3994643467E
:1063600020001A685B68290001F0CEF808235B4220
:106370009C46E04406000F00D045D5D1059B300077
:106380001A003900984600F0DDFCFF2300229B052F
:1063900004000D0001F0DCFC00F038FC0022764B1C
:1063A00001F0D6FC02000B002000290001F042FFA2
:1063B0000D00040002F086FA814602F0B9FA0200EC
:1063C0000B002000290001F035FF060040460F00B9
:1063D000002800DCEEE0009B18215A1E92000EAB54
:1063E0009B58091A1D000D41A9448D405D1B0EAB41
:1063F0009D5017231B1A1D41002D2DDD01239C46A6
:10640000009BE144002B00DC1CE20E9C0123002CCD
:1064100000D0B5E0009A012A09D099000EAA54587C
:106420000133002C00D0ACE0009A9A42F5D1059BD4
:10643000002B0EDD012B00D1A8E1022B09D1009B1E
:106440000EA95A1E92000EAB9B5807939B029B0A03
:106450008B50022D00D1C1E0002300223000390012
:1064600000F07EFE009B002800D194E2069A591E9F
:106470008A4210DC414A0A9894460EAA6344944624
:1064800000229B0063441C68043B22438342FAD1F0
:10649000002A00D0C0E0069B0EAA013B9B00D35807
:1064A000002B00D0B3E001220C9B043B5968013261
:1064B0000029FAD0009B9C466244110007921A0002
:1064C00001338B4246DC0B9863468046A59C4344CF
:1064D000A046099C9B00A1464A449844D30022AAA6
:1064E0009146049A99449446089BA59A634484462D
:1064F000614494469A468B0063440093434658682F
:1065000002F016FA4B4618605960029B002B24DB00
:106510004D46039C0026002701E0286869680CCCE2
:1065200001F016FC02000B003000390000F0ECFF17
:10653000083D06000F005C45EFD153469E60DF60CA
:1065400004239C460433E0449C46009BE144E2441F
:106550009845D3D1079B0093D1E600260027ECE7AE
:1065600094FDFFFF20B4000018FEFFFFFFFFFF1F98
:106570000000703E0000704100002040FFFFFF3F20
:10658000002180225204141B0EAA545000999942F3
:106590000EDD0EA884469B000EAA8900D2586144E5
:1065A0006344CF4800E01A68821A04C38B42FAD1D0
:1065B00001243CE7059B002B06D1009B0EAA013B62
:1065C0009B00D558ED1517E70022C64B300000F0B0
:1065D000EBFD002800D024E100253DE732003B0020
:1065E0000020C14901F026FE06000F00002C00D15A
:1065F00032E7059A0020BC4900F0A4FB02000B0022
:106600003000390001F016FE06000F0024E70122D9
:1066100050E70026002754E64B46059A0793884624
:106620008B000EA9CB58183A08950592002B0DD176
:106630008C464146AD4B43449B006344043B586841
:106640000139183A0028F9D088460592059A0020A9
:10665000A54900F077FB434604000D00002B00DA4B
:1066600005E29E000EAB9C464346DB0066449C461A
:10667000059370AB9946049F67440097306802F019
:1066800057F922002B0001F063FB0022386079608B
:10669000974B2000290001F05BFB083F04000D0030
:1066A000043EB945EAD14AAB03939B4600239A4680
:1066B000069B4246994643460132029204934B465A
:1066C000002B00DAAAE080208A4B009D9846C00586
:1066D000894900260027002408E008239C46083545
:1066E000E044544511DC4346186859682A686B68D1
:1066F00001F02EFB02000B003000390000F004FF17
:10670000013406000F00A145E7DA5B46C0C39B4693
:1067100001239C46009BE244083B0093029B9A4560
:10672000CDD1049B9846A49B022B00DD8EE0002B6C
:1067300037DC1FD1059B00271D00039B00249C46CE
:106740001E006544083E2A686B683800210000F08E
:10675000DBFE083D07000C00AE42F4D1089B002B85
:1067600003D080231B069C4664443A0023000D9905
:106770000A604B600720079B18409B239B009D44A9
:106780003CBC90469946A246AB46F0BD009B0EA984
:106790005A1E92000EAB9B5807935B025B0A8B500C
:1067A00057E64346002B00DA70E100200021DB00B1
:1067B0004AAAD61848AF32687368083E00F0A4FEB3
:1067C000B742F8D1089B002B00D025E10B00020056
:1067D0004A984B990D9C2260636001F02BFD434663
:1067E00007000C00002B13DD01254CAEB14638002C
:1067F0002E0021004C4601360CCC00F085FEA1464F
:10680000B045F7DA089B07000C00002B00D015E11B
:106810003A0023000D998A60CB60ABE70026002781
:1068200073E701239C46009BE1440225002B00DD19
:10683000EBE532003B0000202B4901F0FBFC060099
:106840000F0009E60024F2E54AAB0393A49B032B57
:1068500000D08FE74346002B00DC14E1039ADB00F5
:106860009B46130091465B441E685F68234B43447C
:106870000293DB00994448AB9A464B465C681B6820
:106880001800210032003B000090019100F03CFE16
:1068900004000D0002000B000098019901F0CAFCF1
:1068A0003B00320000F030FE4B469860D9601C601F
:1068B0005D6008235B429C46E14426002F00CA45E8
:1068C000DBD14346012B00DCE3E0039A13005B4479
:1068D0001E685F68029BDB0099464A44904610E0C0
:1068E000FFFFFF000000E03F0000F03FFFFFFF3F21
:1068F0000000703EE0B30000FB21F93FFFFFFF1FE7
:10690000984643465C681B681800210032003B0033
:106910000090019100F0F8FD04000D0002000B0052
:106920000098019901F086FC32003B0000F0ECFD7C
:106930004346039A9860D9601C605D60083B26005E
:106940002F009A42DCD14D4694460026002447464B
:10695000083565442A686B683000210000F0D4FDDA
:10696000083D06000C00AF42F4D1039B4A9F5D68CE
:106970009968D868089B002B65D08022120694463F
:106980000D9B6544604464441F605D609960D860FD
:106990001E615C61EEE69A464B460793059B30000C
:1069A0005A423900089500F0CDF900223A4B060012
:1069B0000F0000F0F9FB002824D0384B00223000F3
:1069C000390001F0C5F901F07DFF52460400950041
:1069D00001F0AEFF0022304B01F0BAF902000B00CB
:1069E0003000390001F026FC01F06CFF0EAA505176
:1069F0000122059B524418339046059393000EAA3A
:106A0000D45023E65346300039009C0001F05AFF71
:106A10000EAB1851D04619E680230D9A1B06CB18F1
:106A2000106053600B0002004A984B9901F002FC81
:106A3000434607000C00002B00DDD5E680231B0633
:106A40009C466444E4E62B003A000D9D2A606B608E
:106A50000A000300AA60EB60320023002A616B6128
:106A600088E6099BDB00009372AB049332E4A49B9D
:106A7000022B00DDE8E6002B00DD92E600D079E68F
:106A8000002700246AE6002600246EE7002000218B
:106A900098E60026340068E7000070410000703E70
:106AA000F0B5CE46474680B587B000920193474A7D
:106AB0004B00814688465B08934207DC41464846C6
:106AC00001F000FF4146031E484666D04A46434651
:106AD0004846414601F03CF904000D0002000B005D
:106AE0004846414601F034F9394A3A4B06000F0056
:106AF0002000290001F02CF9374A384B01F09AFBAD
:106B000022002B0001F024F9354A364B00F0FCFC42
:106B100022002B0001F01CF9334A344B01F08AFBB0
:106B200022002B0001F014F9314B324A00F0ECFC4A
:106B30000E9B02900391002B34D000980199002203
:106B40002D4B01F005F9029A039B0490059130004A
:106B5000390001F0FDF802000B000498059901F0DE
:106B600069FB22002B0001F0F3F8009A019B01F071
:106B700061FB224A04000D00214B3000390001F076
:106B8000E7F802000B002000290000F0BDFC020025
:106B90000B004846414601F04DFB07B00CBC904647
:106BA0009946F0BD02000B002000290001F0D0F84A
:106BB000124A134B01F03EFB32003B0001F0C8F8D3
:106BC0004A46434600F0A0FCE7E7C046FFFF3F3ED1
:106BD0007CD5CF5A3AD9E53DEB9C2B8AE6E55A3E67
:106BE0007DFEB157E31DC73ED561C119A0012A3F03
:106BF0001111813FA6F810110000E03F495555558D
:106C00005555C53F49004B0819007047474AF0B534
:106C10004F4691464B005B0D99444646D6464A4640
:106C2000C0B505000C000E0088460700132A27DCBB
:106C3000002A4BDB3E4B13419A460B005246134051
:106C4000034318D03B4A3C4B2800210000F05CFC79
:106C50000022002300F09EFA002847D0002C04DA1E
:106C600080234A465B031341984446465346002717
:106C70009E43380031001CBC90469946A246F0BDA8
:106C8000332A08DD8023DB009945F4D102000B0094
:106C900000F03AFCEFE7294A94460122634452424D
:106CA000DA4092460242E6D0224A234B28002100D5
:106CB00000F02AFC0022002300F06CFA002815D016
:106CC000002C1EDB534646469F430FE0194A1A4BE1
:106CD0002800210000F018FC0022002300F05AFADE
:106CE000002803D0002C04DB0027002638003100E8
:106CF000C1E76400640825430027002DF6D0104E3C
:106D0000F4E74B46142B0BD03422D21A01239340C4
:106D10005D19BD4208D201239C462F00E044D1E713
:106D2000133B9C46E044CDE72F00CBE701FCFFFF7F
:106D3000FFFF0F009C7500883CE4377EEDFBFFFFF2
:106D40000000F0BF4B0070B55B0D14000A00002B73
:106D50001AD14B005B08034315D0234B002200F0EF
:106D6000F7FF224B9C422DDB0A004B005B0D363BAC
:106D70001F4DE318AB422ADC002B0DDD1D4C1B051B
:106D800022401A43110070BD1B4DAB42F0D10200EE
:106D90000B0000F0B9FBF6E71D00353519DA174B8B
:106DA00002009C4209DD0B001548164900F032F83C
:106DB000134A144B00F0CCFFE5E70B0012481349CF
:106DC00000F028F8104A114B00F0C2FFDBE7020088
:106DD000E9E7084C363322401B0513431900002213
:106DE0000B4B00F0B5FFCEE700005043B03CFFFF77
:106DF000FE070000FFFF0F80FF07000050C30000E8
:106E00009C7500883CE4377E59F3F8C21F6EA501DB
:106E10000000903C30B54A00DB0FDB0752081A43F4
:106E2000110030BD02B4714649084900095C4900AF
:106E30008E4402BC7047C046002243088B4274D384
:106E400003098B425FD3030A8B4244D3030B8B426B
:106E500028D3030C8B420DD3FF22090212BA030C74
:106E60008B4202D31212090265D0030B8B4219D355
:106E700000E0090AC30B8B4201D3CB03C01A524175
:106E8000830B8B4201D38B03C01A5241430B8B42BD
:106E900001D34B03C01A5241030B8B4201D30B03A6
:106EA000C01A5241C30A8B4201D3CB02C01A5241CD
:106EB000830A8B4201D38B02C01A5241430A8B4290
:106EC00001D34B02C01A5241030A8B4201D30B0279
:106ED000C01A5241CDD2C3098B4201D3CB01C01A93
:106EE000524183098B4201D38B01C01A524143099D
:106EF0008B4201D34B01C01A524103098B4201D38B
:106F00000B01C01A5241C3088B4201D3CB00C01AF7
:106F1000524183088B4201D38B00C01A524143086F
:106F20008B4201D34B00C01A5241411A00D2014694
:106F3000524110467047FFE701B5002000F0F0F81D
:106F400002BDC0460029F7D076E7704703460B43E1
:106F50007FD4002243088B4274D303098B425FD352
:106F6000030A8B4244D3030B8B4228D3030C8B427E
:106F70000DD3FF22090212BA030C8B4202D3121264
:106F8000090265D0030B8B4219D300E0090AC30B39
:106F90008B4201D3CB03C01A5241830B8B4201D3E6
:106FA0008B03C01A5241430B8B4201D34B03C01ACF
:106FB0005241030B8B4201D30B03C01A5241C30A47
:106FC0008B4201D3CB02C01A5241830A8B4201D3B8
:106FD0008B02C01A5241430A8B4201D34B02C01AA2
:106FE0005241030A8B4201D30B02C01A5241CDD247
:106FF000C3098B4201D3CB01C01A524183098B4292
:1070000001D38B01C01A524143098B4201D34B017A
:10701000C01A524103098B4201D30B01C01A5241DD
:10702000C3088B4201D3CB00C01A524183088B4264
:1070300001D38B00C01A524143088B4201D34B004D
:10704000C01A5241411A00D20146524110467047BF
:107050005DE0CA0F00D04942031000D340425340C4
:1070600000229C4603098B422DD3030A8B4212D384
:10707000FC22890112BA030A8B420CD389019211B6
:107080008B4208D3890192118B4204D389013AD0F3
:10709000921100E08909C3098B4201D3CB01C01AC8
:1070A000524183098B4201D38B01C01A52414309DB
:1070B0008B4201D34B01C01A524103098B4201D3C9
:1070C0000B01C01A5241C3088B4201D3CB00C01A36
:1070D000524183088B4201D38B00C01A5241D9D24E
:1070E00043088B4201D34B00C01A5241411A00D2CF
:1070F0000146634652415B10104601D34042002BCB
:1071000000D54942704763465B1000D3404201B549
:10711000002000F005F802BD0029F8D016E77047FE
:107120007047C046D0400B1C1141203A03D49C4606
:107130001341184363465242934018437047C04678
:107140008446101C62468C46191C634600E0C0460B
:107150001FB500F095FD002801D40021C8421FBDD5
:1071600010B500F0EDFC4042013010BD10B500F04C
:1071700087FD002801DB002010BD012010BDC046A6
:1071800010B500F07DFD002801DD002010BD0120BC
:1071900010BDC04610B500F00FFD002801DC002036
:1071A00010BD012010BDC04610B500F005FD00283F
:1071B00001DA002010BD012010BDC046F0B5CE465A
:1071C000474615042D0C2E0080B50704140C3F0C07
:1071D0009946030C7E435D43674363437F19340C38
:1071E000E4199C46A54203D980235B029846C44417
:1071F0004B4643435143250C36046544360C240466
:10720000A4195B19591820000CBC90469946F0BD92
:10721000F0B54E4657464546DE46E0B543025B0AAA
:10722000450083B00F1C99462D0EC60F002D57D078
:10723000FF2D24D08020DB00C004184300238146AA
:107240009A469B467F3D7C027A00FB0F640A120E31
:10725000984623D0FF2A4BD0E30080240020E4048A
:107260007F3A1C43AD186B1C474601935346774049
:107270003A000F2B48D87D499B00CB589F46002BE6
:1072800000D085E008339A46063B9B467C027A0094
:10729000FB0FFF25640A120E9846DBD1002C00D0AC
:1072A00090E0524601231A4392460120DBE74C4608
:1072B00058461700022824D0032800D1CFE000222E
:1072C000002301284DD15802D205400AFF07104380
:1072D000384303B03CBC90469946A246AB46F0BD4D
:1072E000002B5BD104239A46033B00259B46AAE76B
:1072F000FF35002C60D1524602231A4392460220E9
:10730000B1E7FF220023DEE74B461B0C9C464B46B1
:107310002604360C180461463300220C6446000C27
:1073200043434E435043544380191A0C121896425B
:1073300003D9802149028C4664441B041B0C1004B1
:10734000C01883015E1EB341800E1843130C1B1935
:107350009B0103431C00230179D5012362081C40D3
:107360001443019A7F32002A4DDD630704D00F23B6
:107370002340042B00D00434230103D53C4B019A55
:107380001C408032FE2ABCDCA3015B0AD2B29AE721
:107390000C239A46093BFF259B4654E7180001F051
:1073A00053FB4A46431F76259A4000236D4291467F
:1073B0002D1A9A469B4646E7524603231A439246A5
:1073C000032050E7200001F03FFB431F2D1A9C4093
:1073D000763D002047E780230027DB03FF2272E78A
:1073E000424666E74C463200584662E780234A46EA
:1073F000DB031A4222D01C4220D123435B025B0AEA
:107400004746FF225FE701239A1A1B2A21DC23004B
:107410000199D3409E318C401A0023005C1EA34189
:1074200013435A0704D00F221A40042A00D0043311
:107430005A0111D49B015B0A002244E780234A468B
:10744000DB0313435B025B0A3700FF223BE7019536
:1074500087E70022002336E70122002333E7802359
:10746000DB0323435B025B0AFF222CE730B40000FE
:10747000FFFFFFF770B500283DD0C317C5185D406A
:10748000C40F280001F0E0FA9E22121A962A07DCA7
:10749000D2B2082833DD083885406802400A23E06C
:1074A000992A0BDD052329001B1AD94003001B3341
:1074B0009D402B005D1EAB4119430D00052801DDE9
:1074C000431F9D402B000F490B406E0709D00F262C
:1074D0003540042D05D004335D0102D59F220B40B9
:1074E000121A9B01580AD2B24002D205400AE407A0
:1074F0001043204370BD002400220020F4E76802FE
:10750000400AF1E7FFFFFFFBF0B54F464646D6467F
:107510000C000903C0B5490A470F5E0039431F0339
:10752000DB0F9C4665007B0A570F1F436D0DE40F70
:10753000760DA146C000B846D200AB1B64457BD097
:10754000002B5FDD002E00D0A4E03E00164300D1EA
:1075500012E15E1E002E00D09EE1871A4346B8421B
:1075600080410125C91A4042091A0B0200D431E1B9
:1075700049024E0A002E00D16EE1300001F064FA9B
:107580000300083B1F2B00DD61E120223900D21AE5
:107590009E40D1409F400E439D4200DD51E15D1B66
:1075A0006B1C1F2B00DD7CE12021C91A3D0030003F
:1075B0008F408840DD40791E8F41310007222843EB
:1075C000D940002507433A40002A09D00F233B4009
:1075D000042B05D03B1DBB42BF417F42C9191F0090
:1075E0000B0200D426E26A1CC64B55056D0D9A426B
:1075F00000D106E1C44AFF080A40530752023B4348
:10760000120B8EE0002B00D0B8E06B1C5B055B0D0D
:10761000012B00DC30E1871A4346B842B641CB1A51
:1076200076429E1B330200D54CE13B003343A1D18F
:1076300000220024002570E0002B00DCE5E0002E95
:1076400000D183E0AF4EB54260D080263604374388
:10765000B846382B00DC3EE1434613431F007A1E38
:1076600097413F1887428041404209180B0200D4DD
:10767000B0E0A44B01359D4200D1C3E0A24A7B0893
:107680000A4001210F401F435108D30707221F431F
:107690003A4099E79B4EB54238D0802636043743AE
:1076A000B846382B00DDDCE01F2B00DC30E11E008B
:1076B0004746203EF740BC46202B04D04026F31A14
:1076C00046469E403243170063467A1E97411F4349
:1076D000CCE0002B00D104E24346134300D159E132
:1076E0004B07C00818438023C9081B03194208D060
:1076F0004546ED081D4204D14346D00859070843CA
:107700002900420FC9007F4D1143C0004B07CA0832
:107710007C49C00803438D4268D012036D05120BEB
:107720006D0D002112031800130B0A0D12051A43E8
:10773000764B2D0513402B435B00E4075B08234386
:1077400019001CBC90469946A246F0BD3E00164367
:1077500012D05E1E002E00D000E1871887428041C3
:1077600041444042091801250B0233D5022585E723
:1077700064463300414610001D00C7E7002D00D0CD
:10778000DAE00C000443F3D05C1C00D19FE15D4CB7
:10779000A64200D12FE1DB43382B00DD66E11F2B31
:1077A00000DD83E120240500E41A0F00DD40D9400C
:1077B000A0404346A7405B1A441EA04198462F4371
:1077C0003843171ABA42924143465242991A6446C4
:1077D0003500CAE607223A40002A00D0F6E64B07F9
:1077E000CA084849FF083B438D4296D1190011430E
:1077F00000D19EE1802109030A431203120B414D7F
:107800008FE71500002200238BE7002B00D0C7E094
:107810006B1C5F057F0D012F00DCF1E0394DAB42A1
:1078200000D1B9E085180A008542894142444942A5
:1078300051180722CF076D082F4349083A401D0011
:10784000C2E607223049ED1A31403A40BCE63E001C
:107850002838864000279FE6380001F0F5F82030F0
:107860008EE6434613431F007A1E9741C71BB8425A
:1078700080414042091A78E60E003B00064313435C
:10788000002D61D1002E00D0F4E0002B00D11BE1CF
:1078900064463900100039E71A4FBB427AD03300F2
:1078A000FFE630001F3DE840202B03D04021CB1ADB
:1078B0009E4037437B1E9F41072207433A400021E9
:1078C000002589E7171A4346BA42B641591A76424B
:1078D0008E1B64464EE61F2B00DDADE0202647469A
:1078E000F61AB740B9461700B246DF404E463E434F
:1078F00037005646B240561EB24117434246DA4060
:107900008918AEE6FF070000FFFF7FFFFFFF0F8033
:1079100020264746F61AB740B9461700B246DF4060
:107920004E463E4337005646B240561EB2411743BC
:107930004246DA40891A99E77F4CA6425BD0802400
:1079400024045B42214327E7002E0CD1002B00D1F9
:10795000CBE0644639001000774DD7E6764FBB4246
:1079600018D0330075E6002B14D04B07C00818431D
:107970008023C9081B03194207D0FC081C4204D10C
:107980007907D0080843E14621004C46420FC90060
:107990001143C000684DB9E61D0000220023C0E677
:1079A000002D5BD10D00054300D1E2E65D1C00D146
:1079B000B0E0614DAE421FD0DB43382B71DC1F2B92
:1079C00000DD96E020250F00ED1AAF40B946070014
:1079D000AA46DF404D463D432F005546A840D940BA
:1079E000451EA84188440743BF189742924151421F
:1079F000414435003AE6644635004146100085E6CC
:107A00000B000343002D00D063E6002BF5D0434666
:107A1000134300D17AE68718874280410722414408
:107A2000404209183A400B0200D4D5E6434B0135D9
:107A30001940C9E5380069E61E004746203EF74078
:107A4000BC46202B04D04026F31A46469E403243C3
:107A5000170063467A1E97411F4302E6364DAE4239
:107A6000CAD080252D045B422943A6E70843411E66
:107A70008841A6E6002B00D148E6871A4346B84263
:107A8000B641CB1A76429E1B33024BD5171A43469A
:107A9000BA429241591A5242891A072264463A4020
:107AA00092E501430F00791E8F419DE71C000F00F6
:107AB000203CE740202B03D04024E31A99400843A0
:107AC000411E884138437CE60022002425E6171A2F
:107AD0004346BA429241591A5242891A64463500C5
:107AE00043E541461000144D10E6802200241203A5
:107AF00080E61D000F00203DEF40BC46202B03D048
:107B00004025EB1A9940084307006346781E8741D9
:107B10001F4369E7871897429B4141445B42C9185C
:107B20003500A3E53B003343CED0072231003A4075
:107B300052E600231A00F4E5FF070000FFFF7FFF75
:107B4000F0B54F464646D6468446C0B58046194EE7
:107B500018030F034D00000B5C0082463F0B6D0DB8
:107B6000C90F9146640DDB0F0120B5420AD0B44223
:107B700003D0A54201D157450CD01CBC9046994674
:107B8000A246F0BD66463E43F7D1AC42F5D154461D
:107B90001443F2D10120C845EFD1994207D0002DFE
:107BA000EBD163461F433800471EB841E5E700208C
:107BB000E3E7C046FF070000F0B54F464646D6460D
:107BC0004D00C0B50E03C90F8A462C491F035C0047
:107BD0008046360B6D0D91463F0B640DDB0F8D42D9
:107BE0001ED08C4216D0002D1ED130438446002C6E
:107BF00001D13A4323D06246002A1AD09A4529D0AF
:107C0000514602200139084001381CBC9046994673
:107C1000A246F0BD39001143E5D002204042F4E70E
:107C20003043FAD1AC420FD0002C0FD13A43E7D009
:107C30000CE00122013B934318000130E5E7634665
:107C40000020002BE1D0DBE73A43E6D19A45D7D1BB
:107C5000A542D5DCA54205DBBE42D1D808D0002024
:107C6000BE42D2D250460123013898430130CCE7BE
:107C7000C845C5D80020C845F4D3C6E7FF070000B3
:107C8000F0B54F464646D6464D00C0B50E03C90F67
:107C90008A462E491F035C008046360B6D0D9146C7
:107CA0003F0B640DDB0F8D4218D08C4211D0002D9C
:107CB00018D130438446002C1ED13A431CD1634670
:107CC0000020002B30D051460220013908400138F5
:107CD0002AE039001143EAD0022025E03043FBD1ED
:107CE000AC4226D0002C26D13A4324D15146022062
:107CF00001390840013817E06246002A0FD09A4542
:107D0000E1D1A54205DBBE42DDD819D00020BE423C
:107D10000AD25046012301389843013004E0012281
:107D2000013B9343180001301CBC90469946A24683
:107D3000F0BD3A43D0D19A45C5D1A542C3DCE0E7B6
:107D4000C845C0D80020C845E3D3EDE7FF070000D1
:107D5000F0B55746DE464E464546E0B5834606003A
:107D60000F03480087B092461D003F0B400DCC0F1B
:107D7000002800D16FE0DE4B984238D08023FF000E
:107D80001B041F43730F3B430193DA4B00279946B3
:107D900000239B46F60081442B0369001B0B5246CF
:107DA0009846490DED0F002900D185E0D04B99424E
:107DB00000D173E04346DA0080231B04134352468C
:107DC000CC48520F84461343524600206144D200EF
:107DD00089442100694000918C46012149448A462A
:107DE0000F2F00D990E0C449BF00CF59BF465B4672
:107DF0003B43019300D06AE1022308270026814615
:107E00009B46C9E732005846019B61460091022813
:107E100000D175E0032800D1FEE1012800D02CE15B
:107E200000230027002600253F032A0D3F0BB348FF
:107E300012053A4302401B051343009A5B00D10729
:107E40005B080B433000190007B03CBC90469946D4
:107E5000A246AB46F0BD5B463B43019300D12FE108
:107E6000002F00D1A5E1380000F0EEFD03000B3B30
:107E70001C2B00DD96E11D22D31A5A460100DA4080
:107E80005E4608398F4013008E403B4301939C4B64
:107E900000271B1A994600239B467DE7414653461F
:107EA0000B4393498C46E144002B00D01AE1022297
:107EB0000220174300228CE7134300D10DE1434613
:107EC000002B00D181E1404600F0BEFD02000B3ADC
:107ED0001C2A00DD72E10100434608398B409846B8
:107EE0001D239A1A5346D3401A0043461343524661
:107EF0008A404946081A824989468144002068E739
:107F00007B4B002700268EE7140C1204120C110084
:107F1000370C3604350C794328008C462E0060431C
:107F20006044834656432100300C804658467943CE
:107F300040440291844506D98846802149028C46F6
:107F4000E044414602913604010C360C00048B4695
:107F500081191E0C1B041B0C0391190079438C46DC
:107F6000280075436544A8465843050C45447743AB
:107F7000A94203D9802149028C466744290C8C46CA
:107F800039000004000C2D042D186144AB44059108
:107F90005946049101990F043F0C080C39005143D4
:107FA0004243904602008C46090C8B4662437C4358
:107FB00044445C44A04503D9802149028846424498
:107FC000210C884661460904090C8C463900594346
:107FD000434370437E430F0CF6182404BE196444D7
:107FE00042448C46B34203D980235B029846404406
:107FF000029B61469846049B370443449B46AB452D
:10800000AD416B420D0405992D0C8C467F196744D8
:10801000FD18A8465D462D19A542A4419346644229
:10802000A446C344DC448F42BF4198459B419345DD
:108030009241A445A4415B427F421F43360C524209
:108040006442BF192243BF18624638184302D20D5A
:10805000039913436A020A43501E82416146ED0DA3
:108060002A434E023243D90100D4B3E0012650081E
:1080700032400243DE0732435B08224C5444002C5A
:1080800062DD510709D00F201040042805D0101DD3
:108090009042924152429B180200D90104D580249B
:1080A0001948E400034054441848844200DD27E79F
:1080B0005E075B02D2081F0B630516435B0DB2E639
:1080C000002399460133042700269B4664E60323D8
:1080D000019781460C279B465EE60122012017434B
:1080E000002276E6032303201F43434671E6C04681
:1080F000FF07000001FCFFFF70B40000FFFF0F80CE
:108100000DFCFFFFFF030000FFFFFFFEFE07000066
:108110000023802700933F030026434B83E6019B07
:108120003200A446584670E6AC466EE680270199B8
:108130003F0339422DD03B422BD11F433F033F0B1E
:1081400000951600384B6EE601252D1B382D00DDFD
:1081500066E61F2D40DC35481C0050441600824066
:108160008440EE40501E824134431443EB4062078A
:1081700009D00F222240042A05D02200141D944267
:10818000804140421B181A023ED5012300270026D9
:1081900049E68027019B3F031F433F033F0B0094A9
:1081A000214B40E603005A46283B9A4000260192A4
:1081B0006DE6584600F048FC203057E60300524672
:1081C000283B9A401300002293E6504600F03CFC06
:1081D00020307BE6CA4650E71F201E004042041BA9
:1081E000E640202D03D0124C5444A3401A43501EA5
:1081F0008241324307260027164009D00F20002372
:10820000104014000428B9D122005E075B021F0B46
:10821000D2081643002306E680273F031F433F038F
:108220003F0B1600004BFEE5FF0700001E04000098
:108230003E040000F8B557464E464546DE460C0063
:108240000903E0B5490A460F5F0031431E03DB0F07
:10825000760A9B46530F3343C84E6500C000E40FB7
:10826000D2006D0DA24681467F0D9C469046B742D6
:1082700000D1B9E05B46012673409B46EE1BA34547
:1082800000D183E0002E63DD002F00D0B1E0634613
:10829000134300D123E1731E002B00D0BAE1861AEC
:1082A0006346B04280410125C91A4042091A0B02B7
:1082B00000D447E149024B0A98464346002B00D1BF
:1082C00089E1404600F0C0FB0300083B1F2B00DDA6
:1082D0007CE120223000D21A4146D0409940020071
:1082E0009E400A439D4200DD6AE15D1B6B1C1F2B13
:1082F00000DD94E1202110003500C91A8E40DA40DB
:108300008840DD40711E8E41110007222843002560
:1083100006433240002A09D00F233340042B05D0F6
:10832000331DB342B641764289191E000B0200D4B8
:108330003DE26A1C914B55056D0D9A4200D119E141
:108340008F4AF6080A40570752023743120B9BE048
:10835000002E00D0C5E06E1C7605760D012E00DCE7
:1083600048E16746861ACB1BB042BF417F42B84600
:108370001F004346FF1A3B00B8461B0200D55FE1D1
:1083800037439AD100220024002579E0002E00DC3A
:10839000FAE0002F00D18DE0784B9D4267D080231A
:1083A00067461B041F43BC46382E00DC52E163467F
:1083B00013435A1E93411E188642804140420918B9
:1083C0000B0200D4BEE06D4B01359D4200D1D2E0DE
:1083D0006B4A73080A4001210E401E435108D3071F
:1083E00007221E43324095E71E00164300D045E7A2
:1083F00040E7624B9D423AD0802367461B041F43EF
:10840000BC46382E00DDEBE01F2E00DC3AE13300E5
:108410006746203BDF403B00202E05D04027BF1B96
:108420006646BE40324390464646721E96413343EE
:10843000DAE0002B00D114E26346134300D168E177
:1084400080234E07C008C9081B030643194208D001
:108450006046C008184204D163460100D2085E0796
:108460001643F3009946C900720F444D11434B4621
:10847000DE08424B4F073743CA089D4200D16EE0E9
:1084800012036D05120B6D0D00211203130B0A0D63
:1084900012051A433B4B2D0513402B435B00E407A9
:1084A0005B082343380019003CBC90469946A2461D
:1084B000AB46F8BD6346134311D0731E002B00D0AA
:1084C00007E186188642804161444042091801252F
:1084D0000B0237D502257BE73E0061469146350009
:1084E000C5E75C46002D00D0E1E00B000343F3D06C
:1084F000731C00D1ACE1214B9F4200D13AE1F34320
:10850000382B00DD6FE11F2B00DD8CE120250E00F4
:10851000ED1AAE40B0460600AA46DE404546354359
:108520002E005546D940A8406346451EA8415B1A17
:108530009C463043161AB242924163465242991AFF
:108540003D00B4E607223240002A00D0E4E60B4B9F
:10855000F6084F073743CA089D4200D090E73B001A
:10856000134300D1A6E180231B031A431203120B0D
:10857000024D89E715000022002785E7FF0700006C
:10858000FFFF7FFFFFFF0F80002E00D0C7E06B1CB6
:108590005E05760D012E00DCF0E0C84DAB4200D147
:1085A000B9E085180A008542894162444942511860
:1085B0000722CE076D082E43490832401D00A9E668
:1085C000BF49ED1A114007223240A3E63200283895
:1085D0008240002686E6300000F036FA203073E64E
:1085E000634613435A1E9341C61AB042804140422B
:1085F000091A5CE60E00674606431743002D5ED15C
:10860000002E00D0F3E0002F00D11EE15C46614651
:1086100091462CE7A94FBE427BD01E00F1E6100028
:108620001F3DE840202B03D04021CB1A9A4016432F
:10863000731E9E410722064332400021002583E736
:10864000161A6346B2428041591A40420B1A9846A4
:108650005C4632E61F2E00DDABE02027BB1B9A46AE
:1086600063465746BB40994613004F46F3401F43AD
:108670003B005746BA40571EBA4113436246F24088
:10868000891898E62027BB1B9A4663465746BB408D
:10869000994613004F46F3401F433B005746BA40EC
:1086A000571EBA4113436246F240891A9CE7834B36
:1086B0009F425FD080252D047342294320E7002E7E
:1086C0000CD1002F00D1D0E05C46614691467B4D35
:1086D000CDE67A4FBE421CD01E0065E6002F18D0B2
:1086E000C0084E0706438020C9080003014208D095
:1086F0006346DC08044204D12100DA46D2085E0752
:108700001643F300994601245346C900720F1143E2
:108710001C406A4DABE61D0000220027B4E6002D88
:1087200059D10B00034300D1D6E6731C00D1B2E04F
:10873000624B9F421ED0F343382B6FDC1F2B00DDB2
:1087400097E020250E00ED1AAE40B0460600AA467E
:10875000DE40454635432E005546A840D940451ECB
:10876000A8418C440643B618964292415142614456
:108770003D0025E63D006146914678E60B00034347
:10878000002D00D055E6002BF5D06346134300D1F1
:108790006DE68618864280416144404209180022F5
:1087A0000B0200D4D0E6464B01351940B2E5B14684
:1087B0005DE633006746203BDF403B00202E05D0BE
:1087C0004027BF1B6646BE40324390464646721E57
:1087D00096413343EFE5394B9F42CBD080252D04A2
:1087E00073422943A8E70843411E8841A2E6002FAF
:1087F00000D13CE66346861ACF1AB0429B415B42E9
:10880000FB1A98461B024ED5161A6346B242924195
:10881000591A5242891A5C4600227BE501430E0038
:10882000711E8E419FE71D000E00203DEE40B046B8
:10883000202B04D04025EB1A994008438146484636
:108840004346411E8841184374E60022002417E67F
:10885000161A6346B2429241591A5242891A3D0091
:1088600025E561469146154D01E68022002412035C
:1088700079E61D000E00203DEE40B046202B04D0CE
:108880004025EB1A9940084381464E464346711EE7
:108890008E411E4367E7861896429B4161445B42C6
:1088A000C9183D008CE547463743CED007224146E4
:1088B000324049E600273A00E6E5C046FF070000DF
:1088C000FFFF7FFF30B5144D0A034B00120B5B0D09
:1088D000C90F0024AB4211DD104CA34210DC8024F0
:1088E000640322430E4CE41A1F2C0CDD0D48C31AFE
:1088F000DA4013005C42002900D11C00200030BD8A
:10890000094BCC18FAE7094DE040AC4663449A4065
:1089100013000343EEE7C046FE0300001D04000001
:108920003304000013040000FFFFFF7FEDFBFFFF97
:1089300070B500282DD0C317C5185D40C40F28009E
:1089400000F082F8154B1B1A5B055B0D0A2815DD3C
:108950000B38854000222D032D0B002110002D0324
:108960000A0D2D0B12052A430D4D1B052A401343FA
:108970005B00E4075B082343190070BD0200290077
:10898000153291400A000B21081AC5402D032D0B0A
:10899000E3E70024002300250022DEE71E04000098
:1089A000FFFF0F804100090E4B1C70B5DBB2460281
:1089B000750AC40F012B14DDE0239B006D07360BF5
:1089C000CB1800210A0D280012051C4D32435B050F
:1089D0002A405B0813435B00E4075B08234319004C
:1089E00070BD002914D1002D1ED0280000F02CF8F5
:1089F0000A281CDC0B232A001B1ADA40030015335B
:108A00009D400F4B12031B1A5B05160B5B0DD8E73D
:108A1000002D06D0320B802636036D071643094B16
:108A2000CFE7084B0026CCE700230026C9E7030068
:108A30002A000B3B9A400025E3E7C046FFFF0F806A
:108A400089030000FF0700001C2101231B0498423A
:108A500001D3000C10391B0A984201D3000A0839CF
:108A60001B09984201D30009043902A2105C401886
:108A70007047C0460403020201010101000000002A
:108A80000000000030B51C00094B05001B6885B0D4
:108A9000D868084B002A01D1074B1A0002920193B3
:108AA00000912B002200054900F020F800F0FAFDAB
:108AB00060000020B0B400001EA40000BDB400009F
:108AC000084B10B50400002B02D0002100E000BFCD
:108AD000054B1868836A002B00D09847200001F0EE
:108AE00005FBC04600000000ECB400000EB403B566
:108AF000010003AB044804CB0068019300F020F9A7
:108B000002B008BC03B018476000002070B5002612
:108B10000C4D0D4C641BA410A64209D1002601F097
:108B2000E7FA0A4D0A4C641BA410A64205D170BD99
:108B3000B300EB5898470136EEE7B300EB5898477F
:108B40000136F2E73002002030020020300200201F
:108B50004002002010B5034B0100186800F06AF8CD
:108B600010BDC0466000002010B5034B010018681E
:108B700000F016F810BDC04660000020002310B5BC
:108B80009A4200D110BDCC5CC4540133F8E7030015
:108B90001218934200D1704719700133F9E70000B1
:108BA00070B50500002910D00C1F2368002B00DAD7
:108BB000E418280000F0A8FF1D4A1368002B05D117
:108BC00063601460280000F0A0FF70BDA34209D9C3
:108BD000216860188342F3D118685B6841182160EE
:108BE000EEE713005A68002A01D0A242F9D91968A9
:108BF0005818A0420BD120680918581819608242F1
:108C0000E0D110685268411819605A60DAE7A04252
:108C100002D90C232B60D5E721686018824203D16A
:108C2000106852684118216062605C60CAE7C04603
:108C300004120020032370B5CD1C9D4308350600A7
:108C40000C2D1ED20C25A9421DD8300000F05CFF6F
:108C5000254A14682100002919D1244C2368002BCF
:108C600003D1300000F02AFB20602900300000F022
:108C700025FB431C2BD10C233000336000F045FF53
:108C800003E0002DDFDA0C233360002070BD0B6899
:108C90005B1B19D40B2B03D90B60CC18256003E0A8
:108CA0004B688C420DD11360300000F02EFF200085
:108CB00007220B30231D9043C31AE7D05A42E250DB
:108CC000E4E763600C00EFE70C004968C3E70323A7
:108CD000C41C9C43A042E1D0211A300000F0EEFAFF
:108CE000431CDBD1C7E7C046041200200812002055
:108CF000936810B5013B9360002B04DA9469A3429A
:108D000007DB0A2905D01368581C10601970080089
:108D100010BD00F0FBFB0100F9E7F8B506000F00FD
:108D20001400D518AC4201D1002007E021783A00A8
:108D30003000FFF7DDFF0134431CF3D1F8BD000024
:108D4000F0B59FB002900F0016000593002805D0E3
:108D500083690493002B01D100F0A4FD7B4B9F425B
:108D60005BD1029B5F68BB891B0762D53B69002B07
:108D70005FD0002306AC6361203363761033A376A3
:108D800035002B78002B01D0252B5CD1AB1B049335
:108D90000CD0320039000298FFF7BFFF431C00D10E
:108DA000C4E06269049B9446634463612B78002BA2
:108DB00000D1BBE0012200235242626002A954327A
:108DC00052186E1C2360E360A3601370A3653178B2
:108DD00005225F4800F07AFE751C002835D1226814
:108DE000D30604D5532302A95B1820211970130759
:108DF00004D5532302A95B182B21197033782A2B31
:108E00002CD0350000210A20E3682A786E1C303A05
:108E1000092A64D900292ED026E04E4B9F4202D168
:108E2000029B9F689FE74C4B9F429CD1029BDF684F
:108E300099E73900029800F0BFFB002899D0012083
:108E400040421FB0F0BD01359BE7414B2268C01A7C
:108E500001238340134323602E00B8E7059B191DAF
:108E60001B680591002B01DB099304E05B42E36082
:108E70000223134323602B782E2B0AD16B782A2BE5
:108E800035D1059B02351A1D1B680592002B2BDB83
:108E90000793324E29780322300000F017FE002895
:108EA00006D04023801B8340226801351343236092
:108EB000297806222A486E1C217600F007FE002839
:108EC0003AD0284B002B25D10722059B073393432B
:108ED000083305936369039A9B18636150E7434322
:108EE00001219B18350090E701235B42D0E7002366
:108EF0000A201A000135636029786E1C303909296F
:108F000003D9002BC5D00792C3E74243012352186F
:108F10003500F1E705AB00933A00134B21000298AE
:108F200000E000BF0390039B0133D3D1BB895B06F4
:108F300000D584E70B9884E705AB00933A000A4B11
:108F40002100029800F080F8ECE7C04644B500002C
:108F5000F0B4000064B5000024B50000F6B40000D1
:108F6000FAB40000000000001B8D0000F7B51500EA
:108F700001938A680B6900900C00934200DA130099
:108F800022002B6043321278002A01D001332B607B
:108F900023689B0602D52B6802332B6006272368C3
:108FA0001F4027D0230043331B785A1E9341226869
:108FB000920630D42200019943320098089EB047AF
:108FC000431C25D0062320682A68E1680340002559
:108FD000042B03D18D1AEB43DB171D40A3682269D4
:108FE000934201DD9B1AED180027BD4220D10020DD
:108FF00010E00137E3682A689B1ABB42D2DD2200E9
:109000000123193201990098089EB047431CF0D102
:1090100001204042FEBD3020E1184331087021009C
:109020005A1C45310978A218433202331170C1E746
:10903000220001231A3201990098089EB047431C70
:10904000E6D00137D1E70000F0B589B004920A00FC
:1090500043320593039002920A7E0C000E9B6E2A07
:1090600000D186E01FD8632A33D008D8002A00D167
:109070008CE0582A4DD0250042352A7030E0642A11
:1090800001D0692AF7D1196825680A1D280629D553
:1090900008681A60002803DA2D23029A40421370F0
:1090A0006B4E0A274FE0732A74D008D86F2A1FD05E
:1090B000702AE0D1202209680A43226003E0752A61
:1090C00016D0782AD7D12200782145321170614E0E
:1090D00022E025001A684235111D196013682B70B3
:1090E000012365E008681A606906D3D500B2D1E7AC
:1090F00019682568081D186008682E0605D5544EA5
:1091000008276F2A1BD00A2719E06D06F7D580B211
:10911000F5E745314E4E0A7018682268011D006857
:109120001960150621D5D30702D520231A432260E2
:109130001027002803D1202322689A4322602300AD
:10914000002243331A706368A360002B58DB0422AB
:10915000216891432160002854D1029D002B5AD0F0
:109160002500337842352B7055E05506DBD580B2AB
:10917000D9E71A680D68101D4969186013682E0632
:1091800001D5196002E06D06FBD519800023029D10
:1091900023614FE01A68111D19601568002162688B
:1091A000280000F093FC002801D0401B6060636839
:1091B00023610023029A13703CE023692A0004997A
:1091C0000398059DA847431C3ED023689B0715D4F0
:1091D000079BE068984239DA180037E02200012343
:1091E000193204990398059EB047431C2CD00135D1
:1091F000E368079A9B1AAB42F0DCE9E70025F7E742
:109200000028ADD0029D3900FDF79CFE735C013D46
:109210002B700028F7D1082F09D12368DB0706D56A
:1092200063682269934202DC3023013D2B70029B6C
:109230005B1B2361059B07AA00932100049B0398F5
:10924000FFF794FE431CB8D10120404209B0F0BDA5
:1092500001B5000012B50000124B10B51C68A36BDD
:10926000002B0FD11820FFF775FC0F4BA063036094
:109270000E4B012243600E4B83600B23838100233E
:1092800002614361A46B0B4A206961690A4BFDF7D7
:1092900095FF012200238018594120616161480037
:1092A000400810BD600000200E33CDAB34126DE6D7
:1092B000ECDE05002D7F954C2DF45158002370B540
:1092C000064C05000800236000F0FAFE431C03D1A1
:1092D0002368002B00D02B6070BDC046BC25002049
:1092E0000CB430B5164B9DB00C1E1D6808DA8B23EC
:1092F00001202B6040421DB030BC08BC02B01847B2
:10930000822302A99B008B810023029008619C426A
:1093100000D0631E8B604B6101235B42CB81209A9E
:1093200021AB2800019300F079FC431C01DA8B2368
:109330002B60002CDFD00023029A1370DBE7C046BD
:10934000600000200EB400B50B499CB01DAB02902C
:109350000690079104910948094904CB05910068DA
:1093600002A9019300F05AFC0023029A13701CB06A
:1093700008BC03B01847C046FFFFFF7F6000002015
:109380000802FFFF02780B78002A03D00130013178
:109390009A42F7D0D01A704703000A7801311A7048
:1093A0000133002AF9D170470023C25C0133002A3F
:1093B000FBD1581E704730B50500002A00D130BDE2
:1093C0000C78013A6B1C2C700131002C05D19A18D5
:1093D0009A42F4D01C700133FAE71D00EDE700005B
:1093E000F0B51F000E0087B00590019102920C9815
:1093F000347800F0EAFA082200194378751C13400B
:1094000036D12D2C36D1B51C74780126002F62D0B0
:10941000102F09D1302C07D120222B789343582BC1
:1094200054D110276C7802352D4B3900F3181800F1
:109430000393FDF787FD04910121002349420200B7
:109440008C4618002100303909291AD80C00A7428F
:1094500023DD591C09D06346824206D302D1049908
:10946000A14202DB0123784320182C780135E9E77B
:109470002E00BCE72B2C01D01E00C7E7B51C74786A
:10948000FAE721004139192901D8373CDFE72100EB
:109490006139192901D8573CD9E75A1C08D1059AD6
:1094A00023331360029B0398002B09D107B0F0BD52
:1094B000002E00D04042029A002AF7D0002B01D0A3
:1094C0006B1E0193029B019A1A60EFE73024002F74
:1094D000AAD10827A8E7302C9ED00A27A4E7C046C7
:1094E000FFFFFF7F37B51300064A05001068046AC6
:1094F000002C00D1044C0A0000942900FFF770FFF3
:109500003EBDC04660000020C4000020F8B5050044
:109510000E001400002804D08369002B01D100F054
:10952000C1F9224B9C422DD16C68A369A360A38929
:109530001B0731D52369002B2ED023682269F7B28F
:10954000981A6369F6B2834205DC2100280000F016
:109550003BF9002826D1A3680130013BA3602368B2
:109560005A1C22601F706369834204D0A389DB0701
:109570001AD50A2E18D12100280000F025F900285C
:1095800012D00FE00A4B9C4201D1AC68CDE7094BE9
:109590009C42CAD1EC68C8E72100280000F00CF812
:1095A0000028CAD0012676423000F8BD44B500003C
:1095B00064B5000024B50000364B70B51D68060088
:1095C0000C00002D05D0AB69002B02D1280000F063
:1095D00069F9314B9C420FD16C680C23E25E93B267
:1095E00019072DD4D90611D409230120336037334C
:1095F0001343A381404270BD284B9C4201D1AC680B
:10960000EBE7274B9C42E8D1EC68E6E75B0713D514
:10961000616B002908D023004433994202D0300006
:10962000FFF7BEFA002363632422A3899343A38137
:1096300000236360236923600823A2891343A38165
:109640002369002B0BD1A0218022A38989009200DD
:109650000B40934203D02100300000F0E1F90123D8
:10966000A289134011D00023A36063695B42A36108
:10967000002023698342BED10C23E25E1306BAD5D3
:1096800040231343A3810138B5E7920700D46369EF
:10969000A360EDE76000002044B5000064B5000061
:1096A00024B5000010B5062000F0E0FB012000F01A
:1096B0001DFD0000F7B58A8905000C00130760D472
:1096C0004B68002B04DC0B6C002B01DC0020FEBD82
:1096D000E76A002FFAD000232E682B6080235B01FD
:1096E000216A1A4034D0606DA3895B0706D5636890
:1096F000C01A636B002B01D0236CC01A0200216AD0
:1097000000232800E76AB847A189431C06D12B68CB
:109710001D2B30D82B4ADA40D3072CD500236360A9
:1097200023692360CB0405D5431C02D12B68002B91
:1097300000D16065616B2E600029C7D023004433DF
:10974000994202D02800FFF72BFA00206063BEE7A1
:1097500001232800B847431CC6D12B68002BC3D077
:109760001D2B01D0162B01D12E60AFE74023A2891B
:109770001343A381ABE740230B430120A381404265
:10978000A5E70F69002FA1D00B680F60DB1B0193C9
:109790000023920700D14B69A360019B002B00DCE2
:1097A00094E7019B3A00216A2800A66AB047002886
:1097B00003DC4023A2891343DFE7019B3F181B1AF8
:1097C0000193EAE7010040200B6970B505000C0029
:1097D000002B01D1002070BD002804D08369002B2C
:1097E00001D100F05FF80B4B9C4209D16C680C2250
:1097F000A35E002BEED021002800FFF75BFFEAE715
:10980000054B9C4201D1AC68F1E7044B9C42EED180
:10981000EC68ECE744B5000064B5000024B5000036
:10982000002310B5040003604360836081814366B8
:10983000C281036143618361190008225C30FFF734
:10984000A6F9054B24626362044BA362044BE362F6
:10985000044B236310BDC046AD9E0000D59E0000A2
:109860000D9F0000399F000010B5024900F08CF8F0
:1098700010BDC046C997000070B568254A1E554303
:109880000E0029007431FFF7D5F9041E08D000211D
:109890002A00016046600C30A0606832FFF777F95B
:1098A000200070BD836913B50400002B28D18364A8
:1098B000C3640365134B144A1B6882620193984288
:1098C00001D101238361200000F020F860602000B6
:1098D00000F01CF8A060200000F018F80022E06002
:1098E00004216068FFF79CFF01220921A068FFF7AF
:1098F00097FF02221221E068FFF792FF0123A36184
:1099000013BDC046ECB4000069980000F8B51C4BCC
:1099100007001E68B369002B02D13000FFF7C2FFB9
:109920004836B4687368013B04D53368002B07D010
:109930003668F6E70C22A55E002D0DD06834F2E7FC
:1099400004213800FFF798FF30600028F0D10C2385
:1099500004003B602000F8BD20000A4B65662560CE
:109960006560A560E36025616561A5610822290045
:109970005C30FFF70CF96563A563A564E564E9E76E
:10998000ECB400000100FFFFF7B50400070000265B
:1099900001914834002C01D13000FEBD6368A568F8
:1099A0000093009B013B009301D52468F2E7AB894B
:1099B000012B08D90E22AB5E013304D029003800F8
:1099C000019B984706436835EBE7EC300068704729
:1099D00070B50E001D000E23C95E96B0140000295C
:1099E00007DA00232B60B3891B0611D48023DB0028
:1099F0000FE06A4600F0D8FA0028F2DBF022019B63
:109A000012021340054A9B185A4253412B60EDE75E
:109A100040230020236016B070BDC04600E0FFFF69
:109A2000F7B502268B8905000C00334206D02300CF
:109A300047332360236101236361F7BD01AB6A46AD
:109A4000FFF7C6FF009907002800FFF7F3F800288A
:109A500008D10C22A35E9A05EFD4032293431E4340
:109A6000A681E4E70F4BAB628023A28920601343F9
:109A7000A381009B20616361019B002B0DD00E230D
:109A8000E15E280000F0A2FA002806D00322A38994
:109A900093431A0001231343A381A0893843A08173
:109AA000CBE7C0466998000082B0002900D101A927
:109AB000101E06D0002B06D013780B601078431EC2
:109AC000984102B0704702204042FAE7C9B28218BA
:109AD000904201D10020704703788B42FBD00130C7
:109AE000F6E710B5884202D98B18984203D30023B9
:109AF00007E08B5C8354013AFBD210BDCC5CC454AC
:109B000001339A42FAD1F8E770477047F8B5070079
:109B10000D001600002905D11100FFF78BF8040095
:109B20002000F8BD002A03D1FFF73AF83400F7E728
:109B300000F072FA2C00B042F2D231003800FFF788
:109B400079F8041EECD029003200FFF717F829003D
:109B50003800FFF725F8E3E7F0B58E6885B0070019
:109B60000C00039201939E423CD890238A89DB002B
:109B70001A4234D00325096923685B1A029363698A
:109B800002985D43EB0F5D19019B6D1001331B18AB
:109B9000AB4200D91D00530532D529003800FFF72C
:109BA00049F8061E09D10C233B6040230120A289FD
:109BB00040421343A38105B0F0BD029A2169FEF72C
:109BC000DDFFA389144A1A4080231343A381029B1B
:109BD0002661F61826606561019EED1AA560019B5D
:109BE0009E4200D9019E320003992068FFF779FF59
:109BF000A36800209B1BA36023689E192660DAE7F8
:109C00002A003800FFF782FF061EE0D121693800E4
:109C1000FEF7C6FFC7E7C0467FFBFFFFF0B59FB06A
:109C2000029005938B890F0016001B0611D50B6956
:109C3000002B0ED14021FEF7FDFF3860386100286F
:109C400005D10C23029A013813601FB0F0BD4023E8
:109C50007B61002306AC6361203363761033A37607
:109C600035002B78002B01D0252B46D1AB1B04935C
:109C70000CD0320039000298FFF76EFF431C00D170
:109C8000AEE06269049B9446634463612B78002BC9
:109C900000D1A5E0012200235242626002A95432A1
:109CA00052186E1C2360E360A3601370A3653178C3
:109CB00005225448FFF70AFF751C00281FD12268AF
:109CC000D30604D5532302A95B182021197013076A
:109CD00004D5532302A95B182B21197033782A2B42
:109CE00016D0350000210A20E3682A786E1C303A2D
:109CF000092A4ED9002918D010E00135B1E7414BAF
:109D00002268C01A01238340134323602E00CEE74C
:109D1000059B191D1B680591002B01DB099304E0CD
:109D20005B42E3600223134323602B782E2B0AD17E
:109D30006B782A2B35D1059B02351A1D1B680592BD
:109D4000002B2BDB0793304E297803223000FFF7DE
:109D5000BDFE002806D04023801B834022680135C9
:109D6000134323602978062228486E1C2176FFF7CA
:109D7000ADFE00283CD0264B002B25D10722059BA9
:109D800007339343083305936369039A9B18636110
:109D900066E7434301219B183500A6E701235B4298
:109DA000D0E700230A201A000135636029786E1C71
:109DB0003039092903D9002BC5D00792C3E74243A4
:109DC000012352183500F1E705AB00933A00114B1F
:109DD0002100029800E000BF0390039B0133D3D120
:109DE000BB890B985B0600D42FE7012040422CE78B
:109DF00005AB00933A00074B21000298FFF724F9C6
:109E0000EAE7C046F0B40000F6B40000FAB400007F
:109E100000000000599B000070B504000D001F29D0
:109E200004D9162303600120404270BD436C002B0F
:109E300004D08A009B181A68002A08D1200000F07C
:109E400031F82A000100200000F01AF8EDE70020A8
:109E5000012AEAD0511C03D1162301302360E4E724
:109E6000002428001C6090472000DEE710B5034B5B
:109E700001001868FFF7D0FF10BDC0466000002049
:109E8000002370B5064C050008001100236000F0A7
:109E9000FFF8431C03D12368002B00D02B6070BD5A
:109EA000BC25002010B500F0E3F810BD70B50C0023
:109EB0000E25495F00F0B8F8002803DB636D1B181E
:109EC000636570BDA389024A1340A381F9E7C046C8
:109ED000FFEFFFFFF8B51F008B8905000C0016008F
:109EE000DB0505D50E23C95E0022022300F080F8B1
:109EF000A389054A28001340A38132000E23E15EA6
:109F00003B0000F02BF8F8BDFFEFFFFF70B50C0031
:109F10000E25495F00F06CF8A389421C03D1054A65
:109F20001340A38170BD802252011343A381606559
:109F3000F8E7C046FFEFFFFF10B50E23C95E00F043
:109F400021F810BD0B1E04D0FF2A04D98A23036018
:109F50008B3B180070470A700123FAE770B50500C3
:109F6000080011000022064C22601A0000F0B6F82A
:109F7000431C03D12368002B00D02B6070BDC0466A
:109F8000BC250020002370B5064C050008002360A6
:109F900000F05EF8431C03D12368002B00D02B6037
:109FA00070BDC046BC250020002370B5064C0500DE
:109FB00008001100236000F053F8431C03D123680C
:109FC000002B00D02B6070BDBC250020002370B595
:109FD000064C05000800236000F052F8431C03D132
:109FE0002368002B00D02B6070BDC046BC2500202C
:109FF00070B50500080011000022064C22601A000E
:10A0000000F04EF8431C03D12368002B00D02B60D6
:10A0100070BDC046BC2500200B1F1B68181F002BFD
:10A0200001DA0B58C018704770B505000800110020
:10A030000022064C22601A0000F03AF8431C03D1BB
:10A040002368002B00D02B6070BDC046BC250020CB
:10A0500058220120014B40421A607047BC25002065
:10A0600058220120014B40421A607047BC25002055
:10A0700058220120014B40421A607047BC25002045
:10A080005822024B00201A607047C046BC250020B1
:10A0900058220120014B40421A607047BC25002025
:10A0A00058220120014B40421A607047BC25002015
:10A0B00058220120014B40421A607047BC25002005
:10A0C000044A1368002B00D1034B181810601800C5
:10A0D0007047C0460C120020C025002058220120E5
:10A0E000014B40421A607047BC250020FEE7C04685
:10A0F000F8B5C046F8BC08BC9E467047F8B5C046E7
:10A10000F8BC08BC9E46704754050000640500007A
:10A110007E050000FC050000340600006A06000011
:10A12000A2060000C8060000040700004607000061
:10A130009C070000E00700004C08000094080000A5
:10A14000BA080000F2080000380900005E090000AB
:10A150008C090000BE090000F60900007A0A000020
:10A16000460B0000BC0B0000280C0000700C000027
:10A17000900C0000B20C00008C0D0000D20D00000D
:10A180005405000054050000540500004A0E00006C
:10A19000B20E0000340F00007A0F0000C20F000062
:10A1A00040100000BE100000061100004C1100001D
:10A1B00082110000C81100000E12000056120000AB
:10A1C000AA1200000813000046130000B01300009C
:10A1D000E61300002E14000076140000BE140000E8
:10A1E000F814000040150000881500005405000018
:10A1F0005405000054050000F0150000261600006C
:10A200005C16000088160000BE160000F416000060
:10A2100054050000540500005405000054050000DA
:10A220002A1700006C1700005405000054050000B8
:10A23000B2170000021800002818000054050000A2
:10A240005405000054050000561800008618000050
:10A25000B6180000E61800001019000046190000AA
:10A260007019000098190000C0190000F0190000D2
:10A27000201A00004A1A0000741A0000A41A0000F4
:10A28000E81A0000540500005405000054050000C1
:10A290005405000054050000181B0000441B00007A
:10A2A000701B00009C1B0000C81B0000FE1B000070
:10A2B000341C00006A1C0000A01C0000CC1C000024
:10A2C000F81C00002E1D000054050000540500007D
:10A2D000540500005405000054050000540500001A
:10A2E000540500005405000054050000540500000A
:10A2F00054050000540500005405000054050000FA
:10A300005A1D0000861D000066616C736500747242
:10A310007565006C697374206F662025642069740C
:10A32000656D73006F626A656374206F6620636C8D
:10A330006173733A20256400537461636B20756EFA
:10A34000646572666C6F7700070000000300000010
:10A3500091A30000611E000099A30000651E00008B
:10A36000A2A300005D1E0000ABA30000691E000058
:10A3700015000000010000000200000004000000C1
:10A38000050000000600000043616C6C696F706599
:10A3900000686173546F6E6500706C6179546F6E04
:10A3A0006500686173536572766F007365745365F9
:10A3B00072766F00496E73756666696369656E745F
:10A3C000206D656D6F727920666F72204D696372C2
:10A3D0006F426C6F636B73206F626A656374206891
:10A3E00065617000496E73756666696369656E7450
:10A3F000206D656D6F727920666F72204D69637292
:10A400006F426C6F636B7320737461636B000D0A32
:10A41000564D2050616E69633A2025730D0A006D18
:10A420006973630034A40000DD2200003DA4000035
:10A4300095220000686578546F496E740073696EE8
:10A440000000000090A400004923000098A4000030
:10A450004D230000A2A400006B230000ABA4000069
:10A4600075230000B6A400007F230000C2A40000F2
:10A4700089230000D3A4000093230000E9A4000076
:10A480005723000002A50000612300006E657400E0
:10A4900068617357694669007374617274576946DD
:10A4A000690073746F70576946690077696669530C
:10A4B0007461747573006D79495041646472657399
:10A4C00073007468696E6744657363726970746958
:10A4D0006F6E00636C6561725468696E6744657382
:10A4E0006372697074696F6E00617070656E645438
:10A4F0006F5468696E674465736372697074696FDD
:10A500006E00617070656E64546F5468696E675058
:10A51000726F7065727479000D0E0F04050C0B0AD2
:10A520000607080904050C0B0A06070809000000C5
:10A53000000008080800080A4A4000000A5FEA5FB5
:10A54000EA0ED92ED36E19324489330C924C924DB7
:10A5500008080000000488080804080484848800AF
:10A560000A448A4000048EC4800000000488000071
:10A570000EC000000000080001224488100C925216
:10A58000524C048C84848E1C824C901E1EC24492B9
:10A590004C06CA525FE21FF01EC13E02448ED12E0D
:10A5A0001FE24488100ED12ED12E0ED12EC4880069
:10A5B0000800080000048004880244880482000E19
:10A5C000C00EC008048244880ED126C0040ED135C6
:10A5D000B36C0C925ED2521C925C925C0ED0101046
:10A5E0000E1C9252525C1ED01C901E1ED01C90104D
:10A5F0000ED013712E12525ED2521C8808081C1FF6
:10A60000E242524C1254981492101010101E113B3A
:10A6100075B131113935B3710C9252524C1C925CA8
:10A6200090100C92524C861C925C92510ED00C826F
:10A630005C1FE4848484125252524C1131312A44FA
:10A64000113135BB7112524C9252112A4484841E2E
:10A65000C488101E0EC808080E10080482410EC2DD
:10A6600042424E048A400000000000001F0804809F
:10A670000000000ED2524F10101C925C000ED01041
:10A680000E02424ED24E0C925C900E06C81C8808F8
:10A690000ED24EC24C10101C92520800080808023C
:10A6A0004002424C10149814920808080806001B37
:10A6B00075B131001C925252000C92524C001C9207
:10A6C0005C90000ED24EC2000ED010100006C804DE
:10A6D0009808080EC807001252524F0011312A4440
:10A6E00000113135BB00124C8C9200112A449800A5
:10A6F0001EC4881E06C48C8486080808080818082A
:10A700000C881800000C83600000000001000000AD
:10A71000020000000300000004000000050000002B
:10A72000060000000700000008000000090000000B
:10A730000A0000000B0000000C0000000D000000EB
:10A740000E0000000F0000001000000012000000CA
:10A750001400000016000000180000001A0000009D
:10A760001C0000001E00000020000000230000006C
:10A7700026000000290000002C0000002F0000002F
:10A7800032000000360000003A0000003E000000E9
:10A7900042000000460000004B0000005000000096
:10A7A000550000005A000000610000006800000031
:10A7B0006F000000760000007D00000084000000B3
:10A7C0008B0000009200000099000000A000000033
:10A7D000A7000000AE000000B5000000BC000000B3
:10A7E000C3000000CA000000D1000000D800000033
:10A7F000DF000000E6000000ED000000F4000000B3
:10A80000FB000000FF00000058A80000B923000072
:10A8100063A80000852800006DA8000099250000AD
:10A820007AA80000B925000081A8000009260000D0
:10A830008AA800005926000096A80000B128000050
:10A84000A7A80000C9270000B4A8000099270000AD
:10A85000646973706C6179006C696768744C6576C3
:10A86000656C006D62446973706C6179006D62445F
:10A870006973706C61794F6666006D62506C6F74BD
:10A88000006D62556E706C6F74006D62447261771A
:10A890005368617065006D625368617065466F72E0
:10A8A0004C6574746572006E656F506978656C53A1
:10A8B000656E64006E656F506978656C53657450A1
:10A8C000696E004E6F7420656E6F75676820726FD9
:10A8D0006F6D206576656E20616674657220636FAA
:10A8E0006D70616374696F6E00436F6D7061637446
:10A8F000656420466C61736820636F6465207374BF
:10A900006F72650A256420627974657320757365BA
:10A910006420282564252529206F662025640042AF
:10A920006164207265636F726420666F756E642067
:10A93000647572696E6720696E697469616C697AA1
:10A940006174696F6E0025642025642025642028C9
:10A95000256420776F726473290025642072656313
:10A960006F7264732C20256420776F7264732C20BF
:10A970006D617849442025642C20636F6D7061639C
:10A9800074696F6E206379636C657320256400536E
:10A9900063726970747320636C65617265640053DF
:10A9A00074617274656400526573746F72656420BB
:10A9B0002564207363726970747300726164696FD7
:10A9C0000000000052AA0000DD3200005FAA000073
:10A9D000493500006FAA0000ED3400007DAA000098
:10A9E000C936000088AA0000F532000098AA0000CD
:10A9F00069330000ACAA000005330000BBAA0000C8
:10AA0000A9380000C7AA000029380000D0AA000019
:10AA1000CD370000DBAA000015370000E6AA0000D1
:10AA200051370000EFAA000085370000F8AA0000A7
:10AA3000193300006E756D626572006E6F6E650091
:10AA40006F74686572007061697200737472696E08
:10AA5000670064697361626C65526164696F006D5F
:10AA600065737361676552656365697665640070D7
:10AA700061636B65745265636569766500706163D7
:10AA80006B657453656E64007265636569766564B1
:10AA9000496E7465676572007265636569766564A1
:10AAA0004D657373616765547970650072656365A0
:10AAB00069766564537472696E670073656E644984
:10AAC0006E74656765720073656E645061697200CB
:10AAD00073656E64537472696E670073657443685E
:10AAE000616E6E656C0073657447726F757000738C
:10AAF0006574506F776572007369676E616C53742B
:10AB000072656E6774680000000000009630077779
:10AB10002C610EEEBA51099919C46D078FF46A7051
:10AB200035A563E9A395649E3288DB0EA4B8DC7971
:10AB30001EE9D5E088D9D2972B4CB609BD7CB17EF1
:10AB4000072DB8E7911DBF906410B71DF220B06AC1
:10AB50004871B9F3DE41BE847DD4DA1AEBE4DD6DD1
:10AB600051B5D4F4C785D38356986C13C0A86B64D1
:10AB70007AF962FDECC9658A4F5C0114D96C0663F1
:10AB8000633D0FFAF50D088DC8206E3B5E10694CD1
:10AB9000E44160D5727167A2D1E4033C47D4044B11
:10ABA000FD850DD26BB50AA5FAA8B5356C98B242F1
:10ABB000D6C9BBDB40F9BCACE36CD832755CDF4571
:10ABC000CF0DD6DC593DD1ABAC30D9263A00DE51A1
:10ABD0008051D7C81661D0BFB5F4B42123C4B35691
:10ABE0009995BACF0FA5BDB89EB802280888055F11
:10ABF000B2D90CC624E90BB1877C6F2F114C685871
:10AC0000AB1D61C13D2D66B69041DC760671DB015E
:10AC1000BC20D2982A10D5EF8985B1711FB5B60630
:10AC2000A5E4BF9F33D4B8E8A2C9077834F9000F70
:10AC30008EA8099618980EE1BB0D6A7F2D3D6D0810
:10AC4000976C6491015C63E6F4516B6B62616C1C00
:10AC5000D83065854E0062F2ED95066C7BA5011B30
:10AC6000C1F4088257C40FF5C6D9B06550E9B712D0
:10AC7000EAB8BE8B7C88B9FCDF1DDD62492DDA1590
:10AC8000F37CD38C654CD4FB5861B24DCE51B53AB0
:10AC90007400BCA3E230BBD441A5DF4AD795D83DB0
:10ACA0006DC4D1A4FBF4D6D36AE96943FCD96E34F0
:10ACB000468867ADD0B860DA732D0444E51D0333D0
:10ACC0005F4C0AAAC97C0DDD3C710550AA410227E0
:10ACD00010100BBE86200CC925B56857B3856F20B0
:10ACE00009D466B99FE461CE0EF9DE5E98C9D92910
:10ACF0002298D0B0B4A8D7C7173DB359810DB42E50
:10AD00003B5CBDB7AD6CBAC02083B8EDB6B3BF9A9B
:10AD10000CE2B6039AD2B1743947D5EAAF77D29D27
:10AD20001526DB048316DC73120B63E3843B649407
:10AD30003E6A6D0DA85A6A7A0BCF0EE49DFF099307
:10AD400027AE000AB19E077D44930FF0D2A3088777
:10AD500068F2011EFEC206695D5762F7CB67658027
:10AD600071366C19E7066B6E761BD4FEE02BD38927
:10AD70005A7ADA10CC4ADD676FDFB9F9F9EFBE8E87
:10AD800043BEB717D58EB060E8A3D6D67E93D1A1C7
:10AD9000C4C2D83852F2DF4FF167BBD16757BCA6A7
:10ADA000DD06B53F4B36B248DA2B0DD84C1B0AAF47
:10ADB000F64A0336607A0441C3EF60DF55DF67A8C7
:10ADC000EF8E6E3179BE69468CB361CB1A8366BC57
:10ADD000A0D26F2536E2685295770CCC03470BBBA7
:10ADE000B91602222F260555BE3BBAC5280BBDB2A7
:10ADF000925AB42B046AB35CA7FFD7C231CFD0B547
:10AE00008B9ED92C1DAEDE5BB0C2649B26F263EC38
:10AE10009CA36A750A936D02A906099C3F360EEB46
:10AE20008567077213570005824ABF95147AB8E206
:10AE3000AE2BB17B381BB60C9B8ED2920DBED5E5E6
:10AE4000B7EFDC7C21DFDB0BD4D2D38642E2D4F136
:10AE5000F8B3DD686E83DA1FCD16BE815B26B9F6C6
:10AE6000E177B06F7747B718E65A0888706A0FFF26
:10AE7000CA3B06665C0B0111FF9E658F69AE62F8E6
:10AE8000D3FF6B6145CF6C1678E20AA0EED20DD7E6
:10AE90005483044EC2B30339612667A7F71660D006
:10AEA0004D476949DB776E3E4A6AD1AEDC5AD6D946
:10AEB000660BDF40F03BD83753AEBCA9C59EBBDE66
:10AEC0007FCFB247E9FFB5301CF2BDBD8AC2BACA16
:10AED0003093B353A6A3B4240536D0BA9306D7CD86
:10AEE0002957DE54BF67D9232E7A66B3B84A61C4A6
:10AEF000021B685D942B6F2A37BE0BB4A18E0CC366
:10AF00001BDF055A8DEF022D416C6C207461736B51
:10AF1000732073746F70706564007630363600206D
:10AF20002573202573004D656D6F727920636C6504
:10AF300061726564004E6F2066726565207461738E
:10AF40006B20656E74726965730000008CAF000041
:10AF50008949000098AF0000A54900009EAF00009D
:10AF6000D5490000A4AF000057490000AAAF000077
:10AF700015470000B4AF0000054A0000BCAF000058
:10AF80004148000073656E736F72730074656D7075
:10AF9000657261747572650074696C7458007469C7
:10AFA0006C74590074696C745A00746F75636852DC
:10AFB0006561640069326352656164006932635798
:10AFC00072697465000000003CB00000894A00000E
:10AFD0004AB000008D4A000053B00000994A0000BA
:10AFE0005DB000009D4A000066B00000A14A00006C
:10AFF0006BB00000A54A000070B00000A94A000034
:10B000007CB00000AD4A000083B00000B14A0000EF
:10B010008CB00000B54A000091B00000B94A0000B1
:10B020009CB00000BD4A0000A6B00000914A00009C
:10B03000B0B00000954A000074667400656E6162ED
:10B040006C65446973706C617900676574576964F5
:10B05000746800676574486569676874007365742F
:10B06000506978656C006C696E6500726563740088
:10B07000726F756E646564526563740063697263B0
:10B080006C6500747269616E676C650074657874D4
:10B0900000746674546F75636865640074667454F4
:10B0A0006F7563685800746674546F7563685900EF
:10B0B000746674546F7563685072657373757265E6
:10B0C0000057656C636F6D6520746F204D69637206
:10B0D0006F426C6F636B732100705F737069202126
:10B0E0003D204E554C4C002F686F6D652F62726F7E
:10B0F0006D61676F73612F2E706C6174666F726D16
:10B10000696F2F7061636B616765732F6672616D24
:10B1100065776F726B2D61726475696E6F6E6F7299
:10B120006469636E7266352F6C69627261726965FB
:10B13000732F5350492F5350492E63707000535052
:10B1400049436C6173733A3A535049436C6173736A
:10B15000284E52465F5350495F547970652A2C201F
:10B1600075696E74385F742C2075696E74385F74FD
:10B170002C2075696E74385F74290000000000008F
:10B1800000000000C54C0000814C0000A74C0000EE
:10B19000B14C0000BB4C0000A54C000000000000BA
:10B1A0000100000002000000160000000400000082
:10B1B0000500000006000000070000000800000075
:10B1C000090000000A0000000B0000000C00000055
:10B1D0000D0000000E0000000F0000001A0000002B
:10B1E0001B0000001400000013000000110000000C
:10B1F00003000000100000001C0000001D00000003
:10B200001E000000120000001500000017000000E2
:10B2100018000000190000000000000000000000FD
:10B220007551000099580000F551000009520000C6
:10B23000FF510000715100006551000015520000DF
:10B2400091510000615100000000000000003043F7
:10B2500000000000000030C3FB21F93FFB21094042
:10B260007CD91240FB2119407A6A1F407CD92240C8
:10B27000BBFD2540FB2129403A462C407A6A2F40ED
:10B280005C4731407CD932409C6B3440BBFD35403B
:10B29000DB8F3740FB2139401BB43A403A463C40F3
:10B2A0005AD83D407A6A3F404C7E40405C4741401E
:10B2B0006C1042407CD942408CA243409C6B44407D
:10B2C000AC344540BBFD4540CBC64640DB8F4740D4
:10B2D000EB584840FB21494083F9A200444E6E00E0
:10B2E000FC291500D1572700DD34F50062DBC000D2
:10B2F0003C999500419043006351FE00BBDEAB00DA
:10B30000B761C5003A6E2400D24D42004906E00004
:10B3100009EA2E001C92D100EB1DFE0029B11C0091
:10B32000E83EA700F535820044BB2E009CE984006E
:10B33000B4267000417E5F00D691390053833900F6
:10B340009CF439008B5F840028F9BD00F81F3B0096
:10B35000DEFF97000F980500112FEF000A5A8B00AF
:10B360006D1F6D00CF7E360009CB2700464FB7001A
:10B370009E663F002DEA5F00BA277500E5EBC70027
:10B380003D7BF100F739070092528A00FB6BEA001F
:10B390001FB15F00085D8D00300356007BFC460046
:10B3A000F0AB6B0020BCCF0036F49A00E3A91D007F
:10B3B0005E619100081BE60085996500A0145F009E
:10B3C0008D40680080D8FF0027734D0006063100CD
:10B3D000CA561500C9A873007BE260006B8CC000E0
:10B3E00000000040FB21F93F000000002D44743EA6
:10B3F000000000809846F83C0000006051CC783B8B
:10B4000000000080831BF0390000004020257A38BE
:10B41000000000802282E336000000001DF3693541
:10B42000020000000300000004000000060000000D
:10B4300008730000B2720000B2720000E0730000F6
:10B44000AE720000AE720000D6730000E073000020
:10B45000AE720000D6730000AE720000E073000010
:10B46000E4730000E4730000E4730000EC73000078
:10B47000087F00000A7E00000A7E0000288100008C
:10B48000047E0000047E000010810000288100007E
:10B49000047E000010810000047E0000288100006E
:10B4A0001E8100001E8100001E8100002C81000012
:10B4B0002C2066756E6374696F6E3A200061737339
:10B4C000657274696F6E2022257322206661696C33
:10B4D00065643A2066696C6520222573222C206CF5
:10B4E000696E65202564257325730A0064000020B9
:10B4F000232D302B2000686C4C006566674546475D
:10B5000000303132333435363738394142434445DF
:10B51000460030313233343536373839616263644E
:10B520006566000000000000000000000000000050
:10B53000000000000000000000000000000000000B
:10B5400000000000000000000000000000000000FB
:10B5500000000000000000000000000000000000EB
:10B5600000000000000000000000000000000000DB
:10B5700000000000000000000000000000000000CB
:10B58000000000004300504F534958002E00002097
:10B590002020202020202020282828282820202083
:10B5A0002020202020202020202020202020208833
:10B5B0001010101010101010101010101010100497
:10B5C00004040404040404040410101010101010E7
:10B5D00041414141414101010101010101010101DB
:10B5E00001010101010101010101101010101010F1
:10B5F00042424242424202020202020202020202AB
:10B6000002020202020202020202101010102000C6
:10B61000000000000000000000000000000000002A
:10B62000000000000000000000000000000000001A
:10B63000000000000000000000000000000000000A
:10B6400000000000000000000000000000000000FA
:10B6500000000000000000000000000000000000EA
:10B6600000000000000000000000000000000000DA
:10B6700000000000000000000000000000000000CA
:10B6800000000000000000000000000000000000BA
:04B6900000000000B6
:08B69400744AFF7F0100000071
:10B69C00FFFFFFFF400600001800000019FCFFFF31
:10B6AC00FFFFFFFF0200000003000000FFFFFFFF91
:10B6BC00000000000100000000000200010000007A
:10B6CC00FFFFFFFF0000000002000000000004006C
:10B6DC0002000000FFFFFFFF00000000030000005D
:10B6EC0000000800030000000A0000000800000031
:10B6FC00640000200000000044B5000064B50000A8
:10B70C0024B5000000000000000000000000000054
:10B71C00000000000000000000000000000000001D
:10B72C00000000000000000000000000000000000D
:10B73C0000000000000000000000000000000000FD
:10B74C0000000000000000000000000000000000ED
:10B75C00000000004300000000000000000000009A
:10B76C0000000000000000000000000000000000CD
:10B77C00000000004300000000000000000000007A
:10B78C0000000000000000000000000000000000AD
:10B79C00000000004300000000000000000000005A
:10B7AC00000000000000000000000000000000008D
:10B7BC00000000004300000000000000000000003A
:10B7CC00000000000000000000000000000000006D
:10B7DC00000000004300000000000000000000001A
:10B7EC00000000000000000000000000000000004D
:10B7FC0000000000430000000000000000000000FA
:10B80C00000000000000000000000000000000002C
:10B81C0000000000430000000000000000000000D9
:10B82C00000000000000000000000000000000000C
:10B83C0000000000459F0000A99A000000000000D5
:10B84C008EB500008CB500001EA400001EA40000E4
:10B85C001EA400001EA400001EA400001EA40000D4
:10B86C001EA400001EA400001EA40000FFFFFFFF8A
:10B87C00FFFFFFFFFFFFFFFFFFFF00000100415331
:10B88C0043494900000000000000000000000000D7
:10B89C000000000000000000000000000000415308
:10B8AC0043494900000000000000000000000000B7
:10B8BC00000000000000000000000000000000007C
:10B8CC00E9000000514C0000994F0000C1540000E9
:04B8DC00C1000000A7
:040000030000503574
:00000001FF
